:1000000000800020BD0100005504000055040000E0
:1000100055040000550400005504000021040000B0
:100020002104000021040000210400005504000008
:1000300055040000210400005504000011040000D4
:10004000550400005504000055040000550400004C
:10005000550400005504000055040000550400003C
:10006000550400005504000055040000550400002C
:10007000550400005504000055040000550400001C
:10008000550400005504000055040000550400000C
:1000900055040000550400005504000055040000FC
:1000A00055040000550400005504000055040000EC
:1000B00055040000550400005504000055040000DC
:1000C00055040000550400005504000055040000CC
:1000D00055040000550400005504000055040000BC
:1000E00055040000550400005504000055040000AC
:1000F000550400005504000055040000550400009C
:10010000550400005504000055040000550400008B
:10011000550400005504000055040000550400007B
:10012000550400005504000055040000550400006B
:10013000550400005504000055040000550400005B
:10014000550400005504000055040000550400004B
:10015000550400005504000055040000550400003B
:10016000550400007107000055040000550400000C
:10017000550400005504000055040000550400001B
:10018000550400005504000055040000550400000B
:100190005504000055040000550400007D130000C4
:1001A000CD13000055140000111500009515000036
:1001B00055040000550400005504000008B54C4BE0
:1001C0004CF220521A804DF628121A8000BF00BF50
:1001D00000F044F9474B4FF010621A60464A9A60AB
:1001E000464ADA60464B1A6812F4807204D14549D7
:1001F0000A604FF4A8521A60434B1A78100703D5CF
:100200001A7842F008021A70404B2A221A70002312
:100210003F4A40499818884204D23F49595899505A
:100220000433F5E73D4A3E4B9A424FF0000302D2B9
:1002300042F8043BF7E73B493B4A5958995004338D
:10024000B3F5DE7FF7D1394B802103F8011B384924
:100250008B42F9D1374B1A60374B0A221A70374B51
:1002600024221A70A02203F8012C354B1A7891072A
:10027000FBD51A78D206FCD41A7802F00C02082AB0
:10028000FAD1304B03221A7040225A702C4B1A7844
:100290009006FBD51A785106FCD52B4B2B4A1A60D9
:1002A00002225A602A4B20221A70254B1B7803F039
:1002B0000C030C2BF9D1274A274B1A60274B4BF61E
:1002C0007F321A60072243F8042C62B60D4B1A687D
:1002D000D20708D5224900221A600A60214A224921
:1002E000116010221A6000F0BFF800F0BFF8FEE7BE
:1002F0000E20054030800440823F04000100002BA6
:1003000010D0034014D0034002D0074000E0074063
:100310006087FF1F0488FF1F50BE00000488FF1F76
:1003200044B3FF1F000000000082FF1F00E400E054
:100330005FE400E008ED00E00050064001400640A8
:10034000064006400440064044800440000003117B
:1003500000400640C01005000480044014E000E0A6
:1003600004D0034000D0034000DD6850FFFFFFFFD2
:10037000FFFFFFFFFFFFFFFFFFFFFFFFFFFFFFFF8D
:10038000FFFFFFFFFFFFFFFFFFFFFFFFFFFFFFFF7D
:10039000FFFFFFFFFFFFFFFFFFFFFFFFFFFFFFFF6D
:1003A000FFFFFFFFFFFFFFFFFFFFFFFFFFFFFFFF5D
:1003B000FFFFFFFFFFFFFFFFFFFFFFFFFFFFFFFF4D
:1003C000FFFFFFFFFFFFFFFFFFFFFFFFFFFFFFFF3D
:1003D000FFFFFFFFFFFFFFFFFFFFFFFFFFFFFFFF2D
:1003E000FFFFFFFFFFFFFFFFFFFFFFFFFFFFFFFF1D
:1003F000FFFFFFFFFFFFFFFFFFFFFFFFFFFFFFFF0D
:10040000FFFFFFFFFFFFFFFFFFFFFFFFFEFFFFFFFD
:10041000024B1A6801321A60704700BF0488FF1F40
:1004200008B50B4C2368580301D500F0A1F92368E7
:10043000590501D500F00EF823681A0501D500F022
:1004400009F8034B1B68DB04EBD500F003F8E8E781
:100450003480044008B5FFF7E3FFFFFF014B102293
:100460001A807047002005407047FFFF08B500F074
:1004700077F803F00BFDBDE808400146014803F0A2
:1004800063B800BF7C3F000010B50023B0FBF2F45E
:1004900002FB1400092894BF30303730C0B2C85472
:1004A00020460CB10133F1E7CA18547022469A4233
:1004B00006DA885CCC5C8C54C8540132013BF6E708
:1004C000084610BD08B5074B1A791206FBD5D8713E
:1004D000054B1B682BB100F0AFFD044B1A680132CD
:1004E0001A6008BD00A006402C8BFF1F308BFF1F39
:1004F0000A2810B5044602D10D20FFF7E3FFE0B251
:10050000FFF7E0FF10BDFFFF08B5054B9B7D2BB942
:1005100000F00EFD013018BF012008BD012008BD0C
:1005200000A0064010B50B4C23681BB100F090FDF5
:1005300000232360084B9A7D12B1D879C0B210BD58
:1005400000F0D0FC411CF5D0044B1A6801321A604F
:1005500010BD00BF308BFF1F00A006402C8BFF1F7B
:1005600008B5104B1A6842F480621A600E4B40F2D4
:1005700013321A604FF451725A600C4B00221A2148
:100580001A70597001219972882119740C21D9703F
:10059000074B1A60074B1A6000F0E0FBBDE808400B
:1005A00000F01ABE3480044040A0044000A0064081
:1005B0002C8BFF1F308BFF1F30BF704730BF704741
:1005C000014B1868704700BF0488FF1F10F1FF300F
:1005D00000D3FBE77047FFFFF0B50C4B0C4C1A78CB
:1005E00042F0020504EBC50682F001027060094882
:1005F0001A700678002E0CBF8827C82786F00106DF
:1006000047EA0141067044F83510F0BD7088FF1FBD
:100610000080FF1FE888FF1F431E032B10B510D872
:1006200072B6094A52F8230048B1416842F82310D3
:10063000064A018832F81340611A22F8131062B694
:1006400010BD002010BD00BF6088FF1F348BFF1F4E
:10065000013803280AD872B6054B53F82030002021
:1006600013B101305B68FBE762B67047002070474A
:10067000B488FF1F10B572B60123174A1A4412F846
:10068000012C12071CD59900144A52F831402CB99C
:1006900002EB431308305860114B09E041F00101AF
:1006A00052F8314064B902EBC103083058600D4B79
:1006B00042F831300C4B1A78013A1A7062B610BD0C
:1006C0000133052BD9D162B6074B00221A70BDE861
:1006D000104000F0ADBB00BF803F00000080FF1F56
:1006E00088004000C8004000DE88FF1F431E032B27
:1006F00030B532D8194A400140F01000104472B6AB
:10070000174CE25C032A09D8DFE802F0160218054C
:100710000830022213E00830042210E01148124A87
:1007200050F8234014B940F8231002E052F8230097
:10073000416042F823100FE0032200E00522E2545A
:1007400010F0080F01F108030A8843600CBF8823EA
:10075000C82343EA0243036062B630BD0080FF1F36
:100760001C88FF1FB488FF1FC488FF1F00BE70478E
:100770002DE9F047A94B1C78E4B261071AD5A84BC4
:100780001B78A3B1A74A117801F0FF0321B1013B07
:10079000DBB2137003B900BEA34A117801F0FF0366
:1007A00029B1013BDBB213700BB900F07FFC9B4B0E
:1007B00004221A7004F0080303F0FF02002B00F07B
:1007C0005E829A4B9A4C1A78D2B215094FEA920778
:1007D00040F0DA8104EBC703596854F83730C3F3AB
:1007E0008303013B0C2B00F2CC81DFE813F08D0179
:1007F0008D01CA01CA01CA01CA01CA01CA01A80100
:10080000CA01CA01CA010D004B688A4D0A688A48AC
:100810006B608A4B2A60012144F837300170884FA1
:1008200092B240F28160002382423B602361A36167
:1008300017D8B2F5D06F80F01D81B2F5817F00F03E
:10084000CF8006D8802A00F0BA80822A00F0BB80D0
:100850002CE140F202339A4200F0D180B2F5A06F51
:100860001CE042F22100824200F04B810ED8B2F52A
:10087000086F00F09E80B2F5106F40F01781AA78E3
:10088000674B6B4E1A7006F180080AE042F2212194
:100890008A4200F0078142F221339A4200F00A8135
:1008A00004E1336A1A0603D5706A083800F0C0FA0A
:1008B00008364645F5D10026B046DFF8B09156F827
:1008C000090028B1D0F804A000F0B2FA5046F8E7C9
:1008D00049F806005B4BDFF89891F05056F8090094
:1008E00028B1D0F804A000F0A3FA5046F8E7564B20
:1008F00049F80600F050554B23F81800544B18F8EF
:100900000320023A032A08D8DFE802F002040204B6
:10091000002200E0012203F8082008F10108B8F1E4
:10092000040F06F10406C8D14A4B00221A700126B2
:100930009946494A494B3244334412F8012C9B00F2
:1009400012F0080F1A704FEA860825D000F052FA0C
:1009500038B104EB461308305860414B44F8383046
:1009600006E099F8003044F83800013389F8003087
:1009700000F040FA48F0010338B104EBC30208303C
:1009800050602E4A44F8332006E044F8330099F8CA
:100990000030013389F8003048F00202013648F097
:1009A00003080023052E44F8323044F83830C0D113
:1009B00081E01B4B2B4C1B7823700B467EE0294CAF
:1009C0002370637079E0AA88042A6FD8254C9200BE
:1009D00023706370244B9B5C9B076ED521706CE089
:1009E000AA8802F07F03042B60DC6B88002B5DD1AA
:1009F00091001D4A0A44117821F0020154E0AA88AE
:100A000002F07F03042B51DC6B88002B4ED1910048
:100A1000154A0A44117841F0020145E08020074060
:100A2000E788FF1F7188FF1FE988FF1F902007409C
:100A30000080FF1FD488FF1FE888FF1FC800400008
:100A40000888FF1F0C88FF1FC488FF1F348BFF1FFF
:100A50001C88FF1FDE88FF1F803F000030C8011088
:100A600088004000DF88FF1FC02007406088FF1F0C
:100A7000B488FF1F6A88A9889E4B53F8084CA3F1DD
:100A80000C009CB133F80C6C964209D133F80A6C17
:100A90008E4205D1120A032A0CBF237803890DE088
:100AA0000C33EAE7A978944A117004E0934B0F22C3
:100AB0001A7026E000231C4600E00223EE88B342B1
:100AC00038BF1E46402E34BF3546402520462946B5
:100AD000FFF782FD761B2C4403D1402D11D1354602
:100AE00003E0402E34BF3546402520462946FFF717
:100AF00073FD761B2C4401D1402D02D1804A3C600D
:100B0000168001227F4B3BE07F4B1A8842F2210383
:100B10009A4210D10023C85C7C4A98540133072BB9
:100B2000F9D11368862B02D1794B0F221A7000205D
:100B30000146FFF751FD774B44F8373021E0764E00
:100B40003568A5B16E4FB7F80080B8F1400F34BFDB
:100B50004446402428462146FFF73EFDC4EB0803E7
:100B60009BB23B800BB9402C00D12B193360664BF4
:100B70001A88B2F5A06F04D100225A709A78674B98
:100B80001A7001225F4B6CE004EBC706013D7368ED
:100B900002F00802A3F10800EDB202F0FF01002A02
:100BA00036D000F045F95E495E4B51F82520EAB198
:100BB000506841F8250002F108017160595D032970
:100BC0000BD8DFE801F002040608032104E002214B
:100BD00002E0052100E00421595516F0080F1288A3
:100BE0000CBF8823C82343EA024342E05A5D032A2C
:100BF00007D8DFE802F040400204002206E00122AC
:100C000004E016F0080F0CBF022203225A5532E00E
:100C100054F83720120C23F8082C22B323F8061CB2
:100C200043F8041C4049DFF830E151F8253013B98E
:100C300041F8250002E05EF8251048603B4B4EF875
:100C4000250033F815100A4423F8152000F0D2F8D7
:100C500010B10830706006E0354B44F837001A7860
:100C600001321A7007E02B4B324A16F0080F08BF0A
:100C7000134644F83730304B08221A707AE5E607FD
:100C800020D520492B482D4C02230B702C4B1A7079
:100C90002C4B186098602C481A61D8609A615C608F
:100CA000164B0D2018702948FF23037000F8083CEC
:100CB0000274274A1370274B9F221A7001230B706E
:100CC000BDE8F087250605D50C4B0D221A70802251
:100CD00003F8402CA00706D51C4B1A78D2B21A7024
:100CE000022203F8082CE10602D5134B10221A70D9
:100CF000BDE8F087903F0000F888FF1FC020074044
:100D0000DC88FF1F94200740D488FF1F3C8BFF1F07
:100D10007188FF1FC80040000888FF1F9820074007
:100D2000B488FF1F1C88FF1F6088FF1F348BFF1FC4
:100D3000DE88FF1F88004000802007402088FF1FBA
:100D40007088FF1F0080FF1F7488FF1F88200740E6
:100D50008C200740842007400C88FF1F08B500F056
:100D600089F800231C4A00219950D0180833882B99
:100D70004160F7D1194B196841F480211960184B73
:100D800080211970187816490006FBD4154BC2F360
:100D900007201870C2F30740120E18751A76124A0F
:100DA000FF231370137202F8703C0B7843F040037A
:100DB0000B7001230021137582F8801013710B4B07
:100DC00070226FF450701A7003444FF400721A606E
:100DD000074B10221A7008BD0080FF1F34800440AA
:100DE0000C2107409C2007408020074049E400E098
:100DF0000821074072B60C4A1168B1FA81F30B2B37
:100E000002D962B6002070474FF00040D84021EA76
:100E10000001116062B6054948225343C8180022F8
:100E2000CA504260704700BF6087FF1F0084FF1FE9
:100E30000C4B4822C31AB3FBF2F30B2B11D80A4A0E
:100E4000127822B1094A12780AB1FFF713BC72B6C0
:100E5000074A4FF0004121FA03F31168194311606A
:100E600062B670470084FF1FDE88FF1FE788FF1F00
:100E70006087FF1F1FB572B6154B70221A70154A96
:100E8000412111700F2102F8011C80221A701A787A
:100E90001206FCD5104B186862B6104B984298BFEA
:100EA0000A2301AC98BF584321460A22FFF7ECFA07
:100EB0000023E15C0A4A29B102EB430001330A2B0B
:100EC0004180F6D101335B00137004B010BD00BF48
:100ED0000000024007000240080002407F96980090
:100EE000EC87FF1F10B5104C23686BB12068428857
:100EF000531C0244147A0288934212D3FFF798FFDE
:100F0000094B00221A600DE0084B1B7813B94FF013
:100F1000FF3010BD0320FFF77FFB20600028E5D1E4
:100F2000F5E74380204610BDF488FF1FE788FF1FC8
:100F300010B50B4C236813B123686BB902E0094B61
:100F40001B7813B94FF0FF3010BD0320FFF764FB8F
:100F500020600028F0D1F5E75A881344187A10BDB4
:100F6000F488FF1FE788FF1F2DE9F8432D4E01236A
:100F700007460C463370002C4FD02B4D2B68A946EA
:100F80002BBB47F20958294B1B7803F0FF020BB922
:100F9000327015E00420FFF75BFB072808D8012317
:100FA0003370FFF727FFC9F8000080B91D4B187098
:100FB000B8F101081E4B01D01A782AB101221A702B
:100FC0004FF0FF30BDE8F883FFF7F8FADBE7296858
:100FD000174A488800231370C0F14002944238BF7A
:100FE000224600F1080C10448C444880A41A934215
:100FF00004D0F85C0CF803000133F8E71F444B8879
:101000003F2B06D940230B800420FFF76FFB002302
:101010002B60084B05221A70ADE734702046BDE8FE
:10102000F88300BFEA88FF1FEC88FF1FE788FF1FD7
:10103000F088FF1FE988FF1F07B502AB012103F805
:10104000010D1846FFF790FF03B05DF804FBFFFFAA
:101050002DE9F041114B1B78F3B1114E114B34685F
:10106000114D01271F7098464CB1638800272F70DF
:10107000042023802146FFF739FB376009E0FFF7A2
:10108000B9FE014620B104202C70FFF72FFB00E0D1
:101090002F70002388F80030BDE8F081E788FF1F3B
:1010A000EC88FF1FEA88FF1FE988FF1F38B50E4B49
:1010B0001B7803F0FF05ABB90C4C216831B14B88AC
:1010C00004200B80FFF712FB256038BDFFF792FE6E
:1010D000014620B10420BDE83840FFF707BB044BB0
:1010E00001221A7038BD00BFEA88FF1FEC88FF1F7D
:1010F000E988FF1F70B5304B1B681A06FBD42F4BD5
:101100001B681B06F7D472B62D4B1A78002A51D0F3
:101110002C4A116856689568D468106931441432B5
:1011200029441268214401441144C1F34E01264A66
:1011300041F400411160D16A166B556B946BD06B12
:101140003144403229441268214401441144C1F31E
:101150004E011E4A41F40041116002F1081214329E
:1011600052F8141C52F8106C52F80C5C52F8084CEF
:1011700052F8040C126831442944214401441144BA
:10118000C1F34E01124A41F400411160D16A166B5D
:10119000556B946BD06B3144403229441268214422
:1011A00001441144C1F34E010A4A41F40041116067
:1011B00000221A7062B670BD24B0034024B00B4008
:1011C000FA88FF1F38B003402CB0034030B0034012
:1011D0002CB00B4030B00B40214B60221A70E12242
:1011E0005A70204B204A1978204B082901D101213F
:1011F00002E00A2907D13921116013221A601C4B21
:1012000019605A600AE00C290CBF35203D2010609F
:1012100012221A601649174B08601A60164B1749BC
:101220001B78174A03B101230B601360154B164A54
:101230001978164B012901D880210BE0042901D827
:10124000842107E0082901D8852103E0102994BFF3
:1012500086218721116019600D4B01221A70704799
:10126000004007400288FF1F08B003400CB0034055
:1012700008B00B400CB00B40FD88FF1F20B00340AE
:1012800020B00B400388FF1F24B0034024B00B4064
:10129000FA88FF1F0D2838B511D9172801D80E3844
:1012A0000CE0A0F11A03DBB2052B01D8093805E0E8
:1012B000A0F12203DBB2062B49D81838C0B2254B67
:1012C0001C5C254B1B780BB1FFF714FF250615D4CA
:1012D00072B6224B1C60224B01221A7062B61D4668
:1012E00072B61E4B1B68180601D51E4B20E02B78EA
:1012F000002BEED062B6FFF761F9F1E772B61A4B38
:101300001A6814F0400F14BF22F0100242F01002CD
:101310001A60164B04F03F021A60154B01221A7036
:1013200062B61D4672B6114B1B68190608D5114BE3
:10133000186800232B7062B60F4B1B78184138BD1C
:101340002B78002BDBD062B6FFF738F9EAE70020F4
:1013500038BD00BFD83F0000FA88FF1F00B003402F
:10136000FC88FF1F10B003400CB00B4000B00B40D6
:10137000FB88FF1F10B00B40F988FF1F114B10B501
:101380001C68E0041C6004D50F4BDA680AB1DB6806
:101390009847A10404D50C4B1A690AB11B699847F8
:1013A000A20604D5084B1A6E0AB11B6E9847E306D5
:1013B00006D5054BD3F8842012B1D3F88430984772
:1013C00010BD00BFA09004400089FF1F1F4B10B547
:1013D0001C68E1031C6004D51D4B1A680AB11B6828
:1013E0009847A20304D51A4B5A680AB15B6898471C
:1013F000E30704D5164B1A6C0AB11B6C9847A0077B
:1014000004D5134B5A6C0AB15B6C9847210704D57D
:101410000F4B9A6C0AB19B6C9847620704D50C4B32
:10142000DA6C0AB1DB6C9847230304D5084B5A6E7B
:101430000AB15B6E9847640306D5054BD3F880204C
:1014400012B1D3F88030984710BD00BFA0A004406F
:101450000089FF1F2C4B10B51C6821071C6004D5A8
:101460002A4B5A6A0AB15B6A9847E20604D5274BB1
:101470009A6A0AB19B6A9847630604D5234BDA6AD5
:101480000AB1DB6A9847200604D5204B1A6B0AB1D3
:101490001B6B9847A10604D51C4B5A6B0AB15B6BBA
:1014A0009847E20704D5194BDA6B0AB1DB6B984712
:1014B000A30704D5154B9A6D0AB19B6D9847600739
:1014C00004D5124BDA6D0AB1DB6D9847A10504D53E
:1014D0000E4BDA6E0AB1DB6E9847E20504D50B4B72
:1014E0001A6F0AB11B6F9847630504D5074B5A6FF3
:1014F0000AB15B6F9847200504D5044B9A6F0AB177
:101500009B6F984710BD00BFA0B004400089FF1F2B
:101510001E4B10B51C68E1071C6004D51C4B9A6873
:101520000AB19B689847220604D5194B5A690AB13B
:101530005B699847E30604D5154B9A690AB19B6924
:101540009847600704D5124BDA690AB1DB699847FE
:10155000210704D50E4B1A6A0AB11B6A9847A207E5
:1015600004D50B4B9A6B0AB19B6B9847A30604D525
:10157000074B1A6D0AB11B6D9847600604D5044BE2
:101580005A6D0AB15B6D984710BD00BFA0C0044002
:101590000089FF1F094B10B51C681C60A30704D508
:1015A000074B9A6E0AB19B6E9847E00704D5044B2F
:1015B000DA6F0AB1DB6F984710BD00BFA0D00440BE
:1015C0000089FF1F212810B518D80D4A52F8303075
:1015D00093F880423CB1012211B183F8802010BD04
:1015E00083F8002110BD02EBC00043681A6811B1F6
:1015F00042F0030201E022F002021A6010BD00BFB7
:10160000F03F0000212806D8044B53F8303093F8FF
:101610000002C0B270470020704700BFF03F0000DA
:10162000212816D80B4A02EBC00301295B6852F847
:10163000302004D182F880124FF4A27208E000201A
:1016400082F8800211B94FF4807201E040F2031277
:101650001A607047F03F000072B60B4B0B491A68D6
:101660000B4B1B68096862B6490102D5322A88BF54
:101670000133C2F53B4230217F32B2FBF1F24FF42D
:101680007A7000FB0320704718E000E004ED00E0F2
:101690000488FF1F38B50446FFF7DEFF054664B136
:1016A000FFF7DAFF401BB0F57A7F03D3013C04D08B
:1016B00005F57A75FEF782FFF2E738BD024B1B781D
:1016C000DB07FBD5704700BF010002404FF400600C
:1016D0007047FFFF7FB5174B6A4603F110066D4652
:1016E00018685968144603C40833B3422246F7D138
:1016F000114B1B78990713D5104B80221A70332297
:101700001A710322DA7072B60D4845F00105A84738
:1017100062B60B4B1A7812F0700201D01A7007E013
:1017200044F62163044A1278D20701D4013BF9D16F
:1017300004B070BD004100000100024007000240FB
:10174000000002404FF0A0507047FFFF08B50E4B5D
:101750001B78D80701D4FFF7BDFF4FF0A0531B78CB
:10176000FF2B0DD06FF06C4303F16C4013F8012F89
:1017700001303AB1054A9342F6D14FF4006001E0DE
:10178000002008BD08BD00BF01000240FF07001493
:10179000B0F5006F10B5044609D2064B1B78DB0785
:1017A00001D4FFF797FF04F1A054207810BD00206A
:1017B00010BD00BF01000240B0F5006F38B504460F
:1017C0000D460FD2084B1B78DB0701D4FFF782FFD1
:1017D00004F1A0542378AB4204D02570BDE8384012
:1017E000FFF76CBF38BD00BF01000240B1F84430C4
:1017F000C31A03D48A6C02EB430070478B6B03EB74
:1018000040007047B1F84430C31A03D48A6C02EB2D
:10181000430070478B6B03EB400070478A6B4B6C47
:10182000821A521003D49A4201DA90B270478A6C3D
:10183000801A03EB600080B27047A1F13003DAB286
:10184000092A01D819460EE0A1F16103DBB2192B78
:1018500001D8573907E0A1F14103DBB2192B94BF3E
:1018600037394FF0FF318142B4BF08464FF0FF30A7
:10187000704738B504462146B0F8CC00FFF7B6FFF4
:1018800021464588B4F89400FFF7B0FF254430F8AE
:10189000020C294601F0A4FEC4F8A45038BDD0F8CB
:1018A000A41010B5044631B1B0F8940001F098FED0
:1018B0000023C4F8A43010BD2DE9F04717460022DC
:1018C000C3F8B020D3F850C0D3F8AC20D3F8B05050
:1018D000954222DA282404FB05C4A6798E4218D149
:1018E00004F107080024A64209D018F80490013436
:1018F00000EB040A1AF801ACCA45F4D009E0996B70
:10190000B1F862011946FFF771FF38600120BDE8A8
:10191000F0870135C3F8B050D8E70020BDE8F08764
:1019200003461A46013311780029FAD1101A70477C
:101930002DE9F04FB1B0D36A0E920A780F90612A68
:101940000C461BD006D8242A09D02D2A18D101F123
:10195000010C91E1692A11D06C2A0FD010E003F13B
:10196000080C58681968CDF820C0802310AA01F02F
:10197000D6FFDDF820C00546634601E01D6804334C
:101980006278612A1BD006D8242A09D02D2A19D1C1
:1019900004F1020C70E1692A11D06C2A0FD011E019
:1019A00003F1080C58681968CDF820C0802310AAEC
:1019B00001F0B5FFDDF820C08246634602E0D3F8AF
:1019C00000A00433A278612A1BD006D8242A09D0AB
:1019D0002D2A19D104F1030C4EE1692A11D06C2A89
:1019E0000FD011E003F1080C58681968CDF820C039
:1019F000802310AA01F093FFDDF820C081466346E2
:101A000002E0D3F800900433E278612A1BD006D8B4
:101A1000242A09D02D2A19D104F1040C2CE1692AB9
:101A200011D06C2A0FD011E003F1080C5868196826
:101A3000CDF820C0802310AA01F071FFDDF820C08E
:101A40008046634602E0D3F8008004332279612A9D
:101A50001BD006D8242A09D02D2A19D104F1050C4F
:101A60000AE1692A11D06C2A0FD011E003F1080CA9
:101A700058681968CDF820C0802310AA01F04FFFE4
:101A8000DDF820C08346634602E0D3F800B004339B
:101A90006279612A1BD006D8242A09D02D2A1CD1AC
:101AA00004F1060CE8E0692A14D06C2A12D014E084
:101AB00003F1080C58681968CDF820C0802310AADB
:101AC00001F02DFFDDF820C00990634605E01A689B
:101AD000099201E0196809910433A279612A1BD0A7
:101AE00006D8242A09D02D2A1CD104F1070CC3E002
:101AF000692A14D06C2A12D014E003F1080C58683B
:101B00001968CDF820C0802310AA01F008FFDDF885
:101B100020C00A90634605E019680A9101E01A683E
:101B20000A920433E279612A1BD006D8242A09D00C
:101B30002D2A1CD104F1080C9EE0692A14D06C2ACD
:101B400012D014E003F1080C58681968CDF820C0D1
:101B5000802310AA01F0E3FEDDF820C00B9063465D
:101B600005E01A680B9201E019680B910433227AA0
:101B7000612A1BD006D8242A09D02D2A18D104F1B5
:101B8000090C79E0692A11D06C2A0FD010E003F11A
:101B9000080C58681968CDF820C0802310AA01F0FD
:101BA000BEFEDDF820C00746634601E01F6804332F
:101BB000627A612A1BD006D8242A09D02D2A18D18E
:101BC00004F10A0C58E0692A11D06C2A0FD010E0F9
:101BD00003F1080C58681968CDF820C0802310AABA
:101BE00001F09DFEDDF820C00646634601E01E6858
:101BF0000433A27A612A1BD006D8242A09D02D2AC0
:101C00001CD104F10B0C37E0692A14D06C2A12D0D5
:101C100014E003F1080C58681968CDF820C080233F
:101C200010AA01F07CFEDDF820C00C90634605E0B0
:101C300019680C9101E01A680C920433E27A612A67
:101C400004F10C0C15D010D8242A15D15868196845
:101C5000CDF820C003F1080410AA802301F05FFE34
:101C600023460D90DDF820C006E0692A01D06C2AD9
:101C700002D11C6804330D940E9CE362099CCDF8DC
:101C800020C001940A9CCDF800B002940B9C0497EC
:101C900003940C9C059606940D9C514607944A4665
:101CA00043460F9C2846A047DDF820C00E9C9CF8B8
:101CB0000010E36A024649B1732909D143F8040CC4
:101CC0001C1FFFF72DFE2346024601E01A6804336D
:101CD0000E9C1046E36231B0BDE8F08F30B50C6861
:101CE00005681B1942EB050202600B6030BD2DE94F
:101CF000F0414FEA124E1F0C96B29BB207FB0EF258
:101D0000026003FB06F203FB0EF30A601A0C1B04CD
:101D100005460C46FFF7E2FF07FB06F3284621467F
:101D20001A0CBDE8F0411B04FFF7D8BF30B50568B9
:101D30000C68AA1A9C422CBF1546551EE31A056072
:101D40000B6030BD0B6810B5D318046834BF002297
:101D50000122144404600B6010BD2DE9FF470668A2
:101D60000B6800969642044688461746019304D3B2
:101D70004FF0FF330360002366E05FEA124A1FFA68
:101D800082F919D11B0C03EB0643B3FBF9F31B04D7
:101D9000036003A902A8FFF7AAFF01A9029A039B07
:101DA0006846FFF7C3FF019A2168B2FBF9F31944B3
:101DB000216009FB132347E04FF6FF73B6FBFAF6E9
:101DC000B6F5803F08BF1E4602A803A93304FFF7FB
:101DD0008EFF684601A9029A039BFFF7A7FF4FEA0F
:101DE0000949009A002A07DA684601A952464B467B
:101DF000013EFFF773FFF4E7BDF8065005EB02451F
:101E00004FF6FF73B5FBFAF53604B5F5803F08BF12
:101E10001D4602A803A93A462B462660FFF767FF36
:101E2000684601A9029A039BFFF780FF009B002BE5
:101E300006DA684601A93A46013DFFF783FFF5E758
:101E400023681D44019B2560C8F8003004B0BDE83C
:101E5000F08770B5044615462B460A680668FFF7FA
:101E600046FF236805FB0635256070BD2DE9F04F60
:101E7000C26A036B1768D3F800A08DB08046161DA8
:101E800003F10409D8F8BC3093B19A4510D3D8F8BF
:101E9000C0309A450CD2D8F8C4300133022BC8F8B0
:101EA000C43005D10023C8F8C430B8F8C84003E0F6
:101EB000BAF800400AF1020ABE2C01F2C78201A062
:101EC00050F824F0C1210000C7210000CB21000000
:101ED000D3210000DB210000E3210000EB21000002
:101EE000F3210000FB210000132200001D2200004E
:101EF000252200002B220000332200003D2200009A
:101F0000412200004D2200005922000065220000FD
:101F10006B2200008722000097220000A52200000B
:101F2000B5220000C1220000D9220000EF220000EB
:101F3000032300000F2300001B2300002D230000BB
:101F40003D2300004D2300005D23000061230000BD
:101F50006D23000079230000892300008D230000F9
:101F60009123000095230000A7230000E92300002F
:101F70007F240000832400008F2400009B240000A5
:101F8000A3240000A7240000B1240000B524000011
:101F9000B9240000C1240000DB240000ED2400006F
:101FA000FB24000009250000172500003F25000044
:101FB0004D250000532500006F25000087250000F7
:101FC000A9250000C1250000012600000D26000003
:101FD000292600002D2600003B2600004D2600008B
:101FE00055260000692600006926000073260000BF
:101FF000BD2400009B260000AD260000BF26000087
:10200000D1260000DD260000F9260000FF26000092
:10201000272700003F2700006127000085270000D8
:10202000B1270000E7270000ED270000FD27000092
:10203000072800008728000099280000A528000034
:10204000B3280000C1280000CD280000DF280000D0
:10205000F32800000B2900002F290000632900004D
:1020600081290000A1290000C1290000E729000002
:10207000F3290000092A0000272A00004D2A000049
:10208000712A00008F2A0000A72A0000B52A00004C
:10209000BF2A0000052B0000752B0000932B0000C9
:1020A000A92B0000BF2B0000CD2B0000012C00004D
:1020B000851E0000372C0000452C0000572C000026
:1020C0008D2C0000B12C0000D32C00000D2D000041
:1020D000352D0000612D000009350000F3270000B8
:1020E000812D00008D2D0000932D00009F2D0000FC
:1020F000AB2D0000B72D0000C32D0000E72D000020
:102100000D2E00003F2E0000692E00007B2E0000E7
:10211000972E0000B32E0000C72E0000252F0000D0
:10212000412F000061300000B3300000BD300000DE
:10213000C7300000D9300000EB300000F93000005B
:102140000D3100001931000025310000313100004F
:10215000373100003D3100005F3100006B3100007D
:10216000BF310000DB310000E93100000332000024
:102170000F3200001B320000273200003D32000009
:102180008332000097320000F73200001333000062
:102190003B3300004B33000057330000793300001D
:1021A00087330000A9330000BF330000D3330000A1
:1021B000DF330000EB330000F73300001934000078
:1021C00088481E2117E3FF435CE6336804361F404E
:1021D00058E6336804361F4354E6336804365F40DC
:1021E00050E6336804361F444CE633680436DF1B80
:1021F00048E6336804365F4344E6002F326806F150
:102200000403BABF7F4222FA07F702FA07F71E4615
:1022100038E63368043643FA07F733E646F8047CB9
:10222000043E2FE6376804362CE6336837601F46D5
:1022300028E646F8047C3768043E23E6043621E6A7
:102240003368376046F8043C043E1BE67268336826
:1022500037607360174615E696E80C0086E888003C
:1022600017460FE656F827700CE656F8271006EBCF
:1022700087032FB153F8042C013F43F80429F8E7F2
:1022800004360F46FEE53346002F3FF4FBAD043E17
:1022900043F8047CF6E549F8047C3768A9F10409A1
:1022A0000436EFE546F8047CD9F80070043E09F1E5
:1022B0000409E7E546F8047CD9F80070043EE1E53E
:1022C0003346A9F1080953F8082BC9F80070C9F87A
:1022D000042077681E46D5E54B4646F8047C53F843
:1022E000087BD9F80420083E32609946CAE546F8D2
:1022F000047CD9F8043046F8083CD9F80070083E50
:10230000C0E5C9F80070043656F8047CBAE546F812
:10231000047CD9F80070043EB4E546F8047CD8F893
:102320005C70331FFF1ABF101E46ABE533680436DE
:10233000BB42ACBF00276FF00007A3E5336804364B
:10234000BB4214BF00276FF000079BE533680436DB
:10235000BB42D4BF00276FF0000793E5FF1791E55C
:10236000002F14BF00276FF000078BE5002FD4BFAC
:1023700000276FF0000785E533680436BB422CBFA9
:1023800000276FF000077DE501377BE5023779E52F
:10239000023F77E53B46301F31463268FFF7A7FC26
:1023A00056F8047C6EE53368002BBDBF5B4233609A
:1023B0004FF0FF340124002FBCBF7F4264423B46F4
:1023C000301F31463268FFF792FC013456F8047C26
:1023D0007FF458AD3368FF435B423360002B08BF86
:1023E00001374FE5114100003446736854F8085B2B
:1023F00083EA050B002DB8BF6D42002B06F1040CDB
:1024000008DAB268DB435242B260002A14BF1A46AF
:102410005A1C7260B268CDF80CC009A80AA92B46F4
:10242000FFF765FC2B4608A80BA97268FFF75FFC55
:1024300008A809A90B9AFFF785FC089BDDF80CC0DA
:102440007360099B6046B36021463A46FFF785FCFE
:102450000A9B20460BA93A460B93FFF77EFCBBF183
:10246000000F09DA7368DA43B3685B42B360002B8C
:1024700014BF1346531C73607768264602E57F102D
:1024800000E5336804369F42B8BF1F46FAE433685C
:1024900004369F42A8BF1F46F4E4002FB8BF7F4216
:1024A000F0E47F42EEE47B883F8847EA0347E9E4B3
:1024B0003F78E7E43F88E5E43F68E3E47F8847440A
:1024C0003888BE2898BFD8F83830414698BF33F8CE
:1024D0001000FFF78BF90746D4E4334653F8082B76
:1024E0003A8012147A8077681E46CBE4334653F85C
:1024F000082B3A7077681E46C4E4334653F8082B1D
:102500003A8077681E46BDE4334653F8082B3A609C
:1025100077681E46B6E4D8F838303068C21AD8F862
:10252000B8309A4204DA0388BE2B01D83B8003E01E
:102530004146FFF773F9388077680836A2E43346DE
:1025400053F8082B3A8077681E469BE4B7F9007071
:1025500098E43B887A8843EA0242334653F8081BE2
:102560000A443A8012147A8077681E468AE43268F8
:1025700071680023BB4203D0585C98540133F9E7DB
:10258000B7680C367EE47368F9183368F8183B4670
:1025900013F1FF3305D37A428C180244E45CD4541F
:1025A000F6E7B7680C366DE471683268FFB2002355
:1025B000934202D05F540133FAE7B7680C3661E406
:1025C000334656F80C1B98685C680023A342C3EBA3
:1025D000070210D0BB420CD01D5C01335A1812F810
:1025E000012C9542F2D001D301274BE44FF0FF3785
:1025F00048E4012746E4171E18BF6FF0000741E4C6
:102600007B1C46F8043C3F78043E3BE43368394683
:102610003B440137013F3FF435AC7A1A1A4412F8B3
:10262000012C202AF6D02DE404372BE446F8047C54
:1026300099E88800043E1F4424E446F8047CD9F855
:102640000C70D9F81030043E1F441BE4BAF9003076
:102650009A4417E41FB9BAF900309A4401E00AF12C
:10266000020A376804360DE4D9F800A009F104091C
:1026700008E438464146FFF7D1F8351D376804466F
:102680002E46BF2C7FF618AC20464146FFF7AEF829
:102690000388BE2BD8BF1C460EE446F8047C01F02C
:1026A0001DFC341F07462646FFF7ECBB46F8047CAA
:1026B00001F01BFC341F07462646FFF7E3BBF8B2C8
:1026C000414601F0E9FB043656F8047CFFF7DABB1B
:1026D00041460A2001F0E0FBFFF7D4BB3568002437
:1026E000BC4205D0605D414601F0D6FB0134F7E7FE
:1026F00077680836FFF7C6BB0237FFF7C3BBD8F8C9
:102700003C30D8F840203B44C8F83C30934237680E
:1027100006F104067FF7B6ABCA481821424601F01D
:10272000CCFBFFF7AFBB30683A4610F8011BCDF881
:102730000080334601F0ABF80746FFF7A3BB3068D3
:1027400039460BAA4346344601F0B3F810B10B9B4F
:10275000336002E0043E44F8047C0746FFF792BB76
:10276000344604362168CDF800803A466068334626
:1027700001F08DF8074600287FF484AB04F10806C9
:10278000FFF780BBD8F880303168002B3FF47AAB7C
:102790007800002383423FF475AB5A5CA2F14104F8
:1027A000E4B2192C9CBF2032D2B25A540233F1E762
:1027B0004B46321D43F804ADC8F82C20C8F8303021
:1027C00039463068424601F076FB431C074600F06C
:1027D0009E86D8F83030D8F82C60D3F800A003F1EA
:1027E0000409FFF74FBBB8F8A0404AE7B8F8984093
:1027F00047E795481B21424601F05FFB46F8047C01
:102800004FF0FF3704E01FB937680436FFF73ABBD3
:10281000D8F88C40E4B9C8F824404046FFF73FF8A8
:10282000D8F8A8304BB1D8F85430C8F8A840C8F848
:102830003C30D8F85830C8F84030D8F85C30C8F888
:102840002C30D8F860300120C8F8303000F065BE78
:10285000D8F86820131DC2F800A0A14504D259F889
:10286000042B43F8042BF8E7D9F80460C8F86C305F
:10287000D9F80030D9F808A0C8F88C30043609F12E
:102880000C09FFF7FFBA46F8047D0020C8F82C6059
:10289000C8F8309000F041BE46F8047C043E0027A2
:1028A000FFF7F0BA46F8047CD8F83C70043EFFF716
:1028B000E9BA46F8047CD8F81870043EFFF7E2BA8B
:1028C00046F8047C043E8427FFF7DCBA043EF8B2E5
:1028D0003146424600F086FE0746FFF7D3BA46F877
:1028E000047C083E3046414600F0A4FE0746FFF750
:1028F000C9BAD8F83C301F803F145F800433C8F851
:102900003C3037680436FFF7BDBA4820D8F83C1091
:1029100000F066FED8F83C300233C8F83C30404640
:10292000FEF7BDFF0023C8F82430FFF7ABBA4046DE
:1029300000F011FF46F8047CD8F83C70BF203946FF
:1029400000F04EFED8F83C300233C8F83C3001238A
:10295000341FC8F824300023C8F8AC302646FFF7EF
:1029600091BABF20414600F084FF4046FEF781FF48
:102970000123C8F824300023C8F8AC30FFF782BA2E
:10298000C020414600F075FFD8F83C301F803F144E
:102990005F800433C8F83C3037680436FFF772BAFA
:1029A000C320414600F065FFD8F83C301F803F143B
:1029B0005F800433C8F83C3037680436FFF762BAEA
:1029C0004146C12000F055FFD8F80430D8F83C202B
:1029D00019141380518004330432C8F83C20C8F81D
:1029E0000430FFF74FBAC220414600F042FFFFF724
:1029F00049BA3446394654F8080B424600F002FF03
:102A000077682646FFF73EBA404600F0A4FEBF2096
:102A1000D8F83C1000F0E4FDD8F83C300233C8F898
:102A20003C30FFF72FBA404600F095FEC020D8F8A2
:102A30003C1000F0D5FDD8F83C300233C8F83C30EB
:102A4000FFF720BA3041000062410000404600F02C
:102A500082FEC120D8F83C1000F0C2FDD8F83C300E
:102A600000225A809A800633C8F83C30FFF70ABA31
:102A7000404600F070FEC220D8F83C1000F0B0FDD7
:102A8000D8F83C300233C8F83C30FFF7FBB9344685
:102A9000394654F8080BC222434600F0DFFE77683F
:102AA0002646FFF7EFB946F8047C043E4FF4006772
:102AB000FFF7E8B9404600F03DFEFFF7E3B9D8F86C
:102AC000A83023B10133C8F8A830FFF7DBB9D8F834
:102AD0002430002B7FF4D6A9D8F83C20C8F8542025
:102AE000D8F84020C8F85820D8F84C200123C8F85E
:102AF0003C208032C8F8A830C8F84020C8F82430FC
:102B0000FFF7C0B9D8F8243023B9D4481821424679
:102B100001F0D3F9D8F8A840002C3FF4B3A9013C48
:102B2000C8F8A840002C7FF4ADA95C20D8F83C1070
:102B300000F056FDD8F85430D8F84C20C8F83C3096
:102B4000D8F85830C8F82440C8F840304B464046C2
:102B500043F8042D46F8047DC8F83030C8F82C60DE
:102B6000FFF784F9D8F82C30D8F830901F681E1D74
:102B7000FFF788B946F8047CBAF800004146FEF732
:102B800035FE341F0AF102050746AA462646FFF71E
:102B900079B9BAF802203AF8043B46F8047C43EAD3
:102BA0000247043EFFF76EB9BAF802203AF8043B38
:102BB00046F8047C43EA0247043EFFF763B946F84F
:102BC000047C3AF9027B043EFFF75CB97520D8F823
:102BD0003C1000F005FDD8F83C4002343846414630
:102BE000C8F83C40FEF71AFE214600F0F9FCD8F880
:102BF0003C300233C8F83C3037680436FFF742B93E
:102C0000D8F83830FA1AD8F8B8309A4202DA388848
:102C1000BE2803D938464146FEF700FED8F83C10DE
:102C200000F0DEFCD8F83C300233C8F83C3037689E
:102C30000436FFF727B93B46043656F8047C002BD0
:102C40003FF420A9D9F80830B3F900A009F10C0924
:102C50009A44FFF717B9334653F8082BBA4206D106
:102C6000BAF90020776892441E46FFF70BB9BF1AE5
:102C700049F8082C49F80C7C49F804AC77680AF14B
:102C8000020AA9F10C091E46FFF7FCB83346A9F168
:102C90000C0953F8082BC9F808A0BF1AC9F804207A
:102CA000C9F8007077680AF1020A1E46FFF7EAB811
:102CB000D9F800300133C9F8003023B1BAF9003037
:102CC0009A44FFF7DFB809F10C090AF1020AFFF78D
:102CD000D9B8D9F80010CB19C9F8003093EA070F1A
:102CE000326806F1040302D497EA010F06D41746AE
:102CF000BAF900201E469244FFF7C4B8174609F1FE
:102D00000C090AF1020A1E46FFF7BCB850464146BC
:102D1000FEF784FD41460446B8F89400FEF766FDD0
:102D20000146204600F05CFC09F1040959F804ACA6
:102D3000FFF7A8B89AF8005054460AEB0503A342DF
:102D400005D014F8010F414601F0A6F8F5E79AF80E
:102D500000000230504400F0FAFC8246FFF792B8BF
:102D6000BAF80000D8F83C1000F03AFCD8F83C3033
:102D70000AF102040233C8F83C30A246FFF782B8D9
:102D800046F8047C371F3E46FFF77CB83E1DFFF730
:102D900079B846F8047C4F46043EFFF773B8B9464D
:102DA000043656F8047CFFF76DB846F8047C4746B5
:102DB000043EFFF767B8B846043656F8047CFFF7C0
:102DC00061B833683A46D10FB1EBD37F06F1040600
:102DD00093FBF7F73FF456A87A4393423FF452A887
:102DE000013FFFF74FB833683A4693FBF7F107FB13
:102DF0001137D10FB1EBD37F06F104063FF442A89F
:102E0000002F3FF43FA81744FFF73CB83346326821
:102E100053F8040FFC0F504390FBF7F2B4EBD07F54
:102E200002FB170106D029B10F447760571E1E46DA
:102E3000FFF728B8716017461E46FFF723B83168C0
:102E4000F80F91FBF7F3B0EBD17F07FB131207D01C
:102E500032B1174437605F1EFFF714B849410000D4
:102E600032601F46FFF70EB83368FF435B423360A2
:102E7000002B08BF0137FFF705B83346B16853F898
:102E8000082B70688C1AC71BB460914238BF013F91
:102E90001E46FEF7F7BF3346B16853F8082B70683B
:102EA00011440744B160914238BF01371E46FEF716
:102EB000E9BF341D30463A462146FEF74EFF3768DB
:102EC0002646FEF7DFBF3268002A34460ADA736806
:102ED000D2435B427360002B14BF1346531C336014
:102EE000012500E00025002FB8BF7F4206F104064F
:102EF000B8BF02353A4620463146FEF72EFF022D76
:102F0000276807D0032D08D0012D7EF4BBAF63687E
:102F10005B4263607F42FEF7B5BF63685B426360FC
:102F2000FEF7B0BF38463178FEF787FC002802DA9A
:102F30000027FEF7A7BF30604FF0FF37FEF7A2BFB4
:102F40006FF06302022FD6F800B0D8F80C30C8F842
:102F5000782021DD9BF80020272A1ED10BEB0702E9
:102F600012F8011C272918D10BF1020300240025B7
:102F7000290241EA146B2002CDF814B00490DDE977
:102F8000040113F8014C01330025934244EA000484
:102F900045EA0105ECD14AE0FFB19BF80020242A64
:102FA0000DD0252A06D0232A0ED1013F0BF1010BAB
:102FB0000A2308E0013F0BF1010B022303E0013F6C
:102FC0000BF1010B102347B19BF800202D2A04D1EF
:102FD000013F0BF1010B012200E00022002400253B
:102FE000002F26DD1BF8011B2E2903D10021C8F874
:102FF00078101AE0184603920293FEF71EFCB0F117
:10300000FF3F8446039A029B13D0D8F87810013111
:10301000C8F87810D917614303FB0511A4FB0345D9
:103020000D4414EB0C0445EBEC75013FD8E700228E
:103030001746D8F87830002BBCBF4FF0FF33C8F8E4
:10304000783012B1644265EB4505346046F8045CA3
:10305000002F40F05E82043E4FF0FF37FEF712BFB4
:10306000D8F80C303468079306F1040B06F1080514
:10307000002F22460ADD14F8011B07980392FEF781
:10308000DCFBB0F1FF3F8446039A02D13260FEF7C9
:10309000F9BE58462946079ACDF80CC0FEF7D9FE6E
:1030A000DDF80CC0584629466246FEF74BFE013F4C
:1030B000DEE74046FEF7DDFBFEF7E4BE4046FEF7E6
:1030C000EEFBFEF7DFBE46F8047C00F0E3FE341FA3
:1030D00007462646FEF7D6BE46F8047C00F0FCFE06
:1030E000341F07462646FEF7CDBE46F8047CD8F8C6
:1030F0003870043EFEF7C6BE46F8047CD8F840702F
:10310000D8F83C30043EFF1AFEF7BCBE46F8047CFB
:10311000043E0227FEF7B6BE46F8047C043E0227B2
:10312000FEF7B0BE46F8047C043EBF27FEF7AABEF9
:10313000BF00FEF7A7BEC24B53F8277056F8041B1A
:10314000C8F83090C8F82C6038464246FEF7F0FBCD
:10315000D8F83090D8F82C600746FEF793BE46F8B2
:10316000047C043E2027FEF78DBE324600231568FE
:103170005068946807950436C11AB94203EB0405F8
:1031800002DA0027FEF77EBE0021C1EB070CBCF17E
:10319000000F0CDDDDF81CB011F80BC0013105EBA0
:1031A000010B1BF801BCE345EFD00133E4E71C44FD
:1031B000C31A946053604FF0FF37FEF763BE384682
:1031C000414600F0BEFB002846F8040C0CBF6FF02F
:1031D00009070027043EFEF755BE3846414600F079
:1031E000A9FE0027FEF74EBE39463068424600F081
:1031F000A2FE002830600CBF6FF009070027FEF721
:1032000041BE904B043E33600027FEF73BBE46F8BC
:10321000047C043E0027FEF735BED8F8343053F85E
:103220002770FEF72FBE3346D8F8342053F8081B1A
:1032300042F8271077681E46FEF724BEBB00D8F878
:103240003420C3EB090343F8042C43F8089C002204
:10325000C8F83430BA4207DA56F82200D8F83410E9
:1032600041F822000132F5E727EAE77706EB870706
:10327000754A3E1DA3F10C093F6843F80C2CFEF77C
:1032800001BED8F83430D9F8009053F8043CC8F89F
:103290003430FEF7F7BDD8F8AC30D8F850402825C8
:1032A00005FB03FB04EB0B03414638460293FEF794
:1032B000B5FA029B3268988044F80B20D8F8AC30FD
:1032C00005FB034273689371D8F8AC30B16805FB15
:1032D0000344E01DA27900239A4203D05C5CC454ED
:1032E0000133F9E7D8F8AC300133C8F8AC30F768EF
:1032F0001036FEF7C7BDD8F8502046F8047CD8F841
:10330000B03028214B43D118D7588C88043EFFF7A2
:10331000B8B9D8F83820D8F83C30CDF80080D8F8C3
:1033200004103446019154F8080B39469B1A00F0FA
:10333000DFFD77682646FEF7A5BD38463146424692
:1033400000F0E4FD0746FEF79DBD46F8047C043E10
:103350000027FEF797BD3446706821683A46434619
:1033600000F0CEFD002806F1040660600CBF6FF08F
:103370000A070027FEF786BD3846414600F0C4FD27
:103380000746FEF77FBDC8F84870D8F83C0034689F
:103390004146FEF743FA351DC8F83C70C8F84400B2
:1033A00027462E46FEF76EBD341D31683A4620464C
:1033B000434600F0B1FD26460746FEF763BD706840
:1033C00056F8081B3A46434600F0ABFD0746FEF7A9
:1033D00059BD46F8047C043E0127FEF753BD46F86C
:1033E000047C043E0227FEF74DBD46F8047C043EF3
:1033F0000427FEF747BD3446706821683A464346C5
:1034000000F080FD002806F1040660600CBF6FF03C
:103410000A070027FEF736BD96E80600FFB2301F08
:1034200000238B4202DA9C5CBC4207D11A44336011
:1034300046F8042CCF1A0646FEF724BD0133F0E708
:1034400014BE000010410000E0410000414620464B
:10345000FEF7CCF90246034632F8020BA0F1BF0199
:10346000082941D8DFE801F0050C151C22292E356A
:10347000380049F804AC9246A9F10409FEF702BDF0
:1034800046F8047C9F885B88043E43EA0747FEF7C2
:10349000F9BC46F8047C5F88043E4744FEF7F2BC62
:1034A00046F8047C1746043EFEF7ECBC46F8047C64
:1034B0005F88043E4744FEF7E5BC5B8838F803406C
:1034C000FFF7DFB8204608F1D00100F089F8FEF7D9
:1034D000D9BC9047FEF7D6BC5B8846F8047C58F808
:1034E0000370043EFEF7CEBC46F8047C414649F822
:1034F00004AC1746FEF77AF9341FA9F10405824699
:10350000A9462646FEF7BEBC4FF0FF3005E002207C
:1035100003E004360027FEF7B5BC0DB0BDE8F08F20
:1035200013B50C46FEF77AF95C23ADF80630236B31
:10353000ADF804001A1F226301AA43F8042C2046A8
:10354000FEF794FC02B010BD37B50C460546FEF7F9
:10355000E7F901AA01462346284600F0AAF9A0B9D6
:103560000C2122460C4800F0A8FC2846FEF7D8F9AA
:1035700022460146284600F0A0FC084802212246C7
:1035800000F09BFC6FF0010003E001982146FFF77B
:10359000C7FF03B030BD00BF7E4100008B4100007B
:1035A00030B5049C039DE363A5F1100323632366F8
:1035B000A5F54C73E366A366A5F55073E362E36576
:1035C000A5F5AA63E364A5F2D453A5F21475646665
:1035D000A063A1646264A36123622565256430BD94
:1035E000088070472DE9F0411546136AAE68D2692C
:1035F0001E44074603EB020834460E60444505D3DB
:103600002B6AE31AAB60A01BBDE8F08114F8013B04
:10361000BB4206D12B6AE31AA41BAB60601EBDE857
:10362000F081202BEADC202FE8D100F033FC0028C9
:10363000E4D1EFE7F0B50C6A8E68CD6926442544E5
:103640003246AA4204D3121B8A6006600020F0BDF5
:10365000134613F8017B202F01DC1A46F1E70260C4
:10366000AB4203D31C1B8C60981AF0BD13F8010BFE
:103670002028F5DC1C1B9B1A8C60581EF0BD2DE920
:10368000F041069C1F46538806460D46E05A2146E7
:10369000FEF7B8F8D4F83880404525D010F8033C40
:1036A00003F03F039D4219D16FF00202521B8318B1
:1036B0000022AA4208D0995C013206EB020C1CF8E9
:1036C00001CC8C45F5D009E0386010F9030C0028D6
:1036D000ACBF4FF0FF300120BDE8F08130F8020CA4
:1036E0002146FEF78FF8D7E70020BDE8F081FFFF05
:1036F0007FB5D36F06460D461446B3B1B2F8CC0081
:103700001146FEF77FF8009402462946304603AB87
:10371000FFF7B5FF48B130462946224600F0CDFB01
:1037200003480E21224600F0C8FB04B070BD00BF64
:103730008E41000008B50146B0F89400FEF762F82B
:1037400010F8033C63F07F0300F8033C08BD013030
:1037500020F001007047C26B10B5511C21F001012F
:10376000891A00238B4203D000249C540133F9E7CB
:103770001344C36310BD2DE9F0410E461C460746B5
:1037800018469046FFF7E7FFF207E36B02D40022EA
:103790001A7001330025B54203DA7A5D5A550135B6
:1037A000F9E726EAE67019181E54CB1CA1F801802F
:1037B000A16BE363591A4910626C03D4914201DA98
:1037C0008BB204E0A16C5B1A02EB63039BB2A4F81A
:1037D0009430BDE8F081D3F8803030B58BB120292A
:1037E000A8BF202100238B420AD0C45CA4F141056C
:1037F000EDB2192D9CBF2034E4B2D4540133F2E76A
:10380000104630BDF0B50D4689B007461146B2F8F6
:10381000CC001446FDF7F6FF234646882946384675
:103820006A46FFF7D8FF294607462246FFF760FFA2
:103830002946A25B23463846FFF79DFFE16BA36B49
:10384000626CCB1A5B1001D4934203DBA36CCB1ADE
:1038500002EB63039BB2A35309B0F0BD38B51C461D
:1038600015461A46FFF7CEFFE36B23F8025BE363CE
:1038700038BD37B5054601A80C46FFF7DBFE2A46E2
:10388000014623460198FFF7E9FF03B030BDF0B5CC
:103890008BB00F46109C16461D4602AA2346FFF722
:1038A0009AFF0094394632462B46FFF7E8FE0BB0EC
:1038B000F0BD2DE9F04F8DB0914604AA88461C4614
:1038C000FFF789FF41464A4623468246FDF7F4FF4B
:1038D000064600BB04F1CE0704F1EE0B034637F8B1
:1038E000020F03932146FDF78DFFA26B039B9042CD
:1038F00005460AD0984209D00094504641462A46CF
:103900004B46FFF7BCFE08B104E01D465F4502D000
:103910002B46E4E7064630460DB0BDE8F08F10B503
:10392000445C6CB1013B994228BF194600238B428D
:1039300003D0C45CD4540133F9E70021D1541046BC
:1039400010BD08B5023000F0F1FA013020F001009E
:1039500008BD7047F8B5174F174B3A681B689A4275
:103960000D4626D2154E316899423CBF0131316077
:103970003368511C03F1FF3E71451C4605D813F80E
:10398000021C03F8011C7346F3E7396010702946E6
:1039900000F082FA33689C4202D214F8010BF6E779
:1039A0003B689C4205D90820294600F075FA013C85
:1039B000F6E7F8BD8889FF1F9489FF1F9889FF1FCC
:1039C000F8B5164A164D12682B689342044624D95E
:1039D000144E013B2B6033680820013B21463360C5
:1039E00000F05AFA2B6837463A68934203F1010611
:1039F00006D258782146187000F04EFA3346F3E7A5
:103A00002020214600F048FA2B689E4205D9082064
:103A1000214600F041FA013EF6E7F8BD8C89FF1F10
:103A20008889FF1F9889FF1FF8B505460D4C0E4B7E
:103A3000226819688A4227461E4607D2107829460E
:103A400000F02AFA236801332360EFE7074B3A6856
:103A50001B689A4203D92846FFF7B2FFF6E73360A6
:103A6000F8BD00BF8889FF1F9889FF1F8C89FF1F41
:103A70000D4A0E491368104613B1B3F5C87F01DD36
:103A8000002308E00023CA56002AF9DB0133B3F50E
:103A9000C87FF8D170470022CA540133B3F5C87FFC
:103AA000F9D10260704700BF9089FF1F9C89FF1FFA
:103AB0001D4B1B68F0B5002B33D01C4A044613463F
:103AC00016461D78E5B99A1A8A4214D1013B9C1B0F
:103AD0008C421A4603F1FF3303DD4A429A5C5A7066
:103AE000F5E7002313708B4203DAC25CF254013312
:103AF000F9E70120F0BD0E4A013393420CD110E0EA
:103B00002778AF4203F1010301D1013406E01A46E0
:103B100001331478002CFAD104461A46044DAB4206
:103B2000CFD30020F0BD00BF9089FF1F9C89FF1FED
:103B30002C8BFF1F38B50C460546FFF799FF3CB3A9
:103B400028462146FFF7B4FF10BB611CB1F5C87FC2
:103B5000A8BF4FF4C8714FF4C873013B8B420D4AA4
:103B600003DB501AC05CD054F7E7002082F88F01C5
:103B7000D054013B01D4E85CFAE7074B1A681144C2
:103B8000B1F5C87FC8BF4FF4C8721960C8BF1A60CA
:103B900038BD00BF9C89FF1F9089FF1FF8B50546FF
:103BA0000E46FFF765FF154B1B6813B3002D20DB96
:103BB000134C00222146AA4208D014F8010B002819
:103BC000FBD1671A9F4217DA0132F4E73046FFF75C
:103BD0002BFF00250B4B1A680B4B1B68D31A013BBC
:103BE0009D4208DA605D30B13146FFF7B3FE013522
:103BF000F0E70020F8BD0120F8BD00BF9089FF1F4D
:103C00009C89FF1F9489FF1F8C89FF1F10B5074AED
:103C1000074C126823689342014605D9082000F03A
:103C20003BF92368013B236010BD00BF8C89FF1F57
:103C30008889FF1F10B5074A074C12682368934212
:103C4000014605D2187800F027F923680133236074
:103C500010BD00BF9889FF1F8889FF1F2DE9F84F0D
:103C6000864B874F18601546864A386001440646E1
:103C7000106085484FF0FF380160002491469A4655
:103C800000F02CF9012C04D15B280CBF0224002485
:103C9000F6E7022C29D1A0F13202162A2CD8DFE84F
:103CA00002F012152B0C2B2B2B2B2B2B2B2B2B2B16
:103CB0002B181B1E212B292B0F006FF01904DFE797
:103CC0006FF0180018E06FF01804D9E76FF01704D0
:103CD000D6E76FF013000FE06FF014000CE06FF008
:103CE000160009E06FF0150006E02CB17E2804D024
:103CF0000024C5E76FF019000446052C6BD025DCC5
:103D000014F1150F00F0848011DC14F1180F56D057
:103D100006DC14F11A0F5ED014F1190F42D099E0AD
:103D200014F1170F60D014F1160F44D092E0012C5B
:103D300038D006DC14F1140F67D0631C00F09280B9
:103D400088E0022C37D0042C39D083E00E2C5FD0D1
:103D50000BDC0A2C1BD003DC062C45D0082C14E00D
:103D60000B2C45D00D2C12D074E0172C62D007DC40
:103D7000102C4AD0152C6DD12846FFF755FEB7E719
:103D80001B2C01D101247BE77F2C05D062E0294662
:103D90000A2000F081F865E03A68DAF800309A42CB
:103DA000A6D914E03A68DAF800309A42A0D9284639
:103DB000FFF72CFFF6E72846FFF728FF98E73A6859
:103DC000D9F800309A4293D22846FFF733FF2846AD
:103DD000FFF7F6FD8CE73A68D9F800309A4287D2AF
:103DE0002846FFF727FFF6E72846FFF723FF7FE780
:103DF0003A68D9F800309A42BFF47AAF2846FFF704
:103E000019FF2846FFF7DCFDF2E708F1010B01E09E
:103E100008F1FF3B58462946FFF7C0FE0024A042A8
:103E200018BFD8462CE713F8013C202B0ED12846AA
:103E3000FFF7C6FD3B68B342F5D807E013F8013C35
:103E4000202B3FF455AF2846FFF7BAFD3B68B3423D
:103E5000F4D84DE71F2C7FF74BAFE0B22946FFF7B0
:103E600079FD45E7D9F80040DAF80030E41A304629
:103E70002146FFF75FFE2046BDE8F88F8C89FF1FC3
:103E80008889FF1F9889FF1F9489FF1F4FF40050F6
:103E900000F054B8012070470A2801D00D2805D140
:103EA00000230B674B6F01334B6702E00B6F01334D
:103EB0000B67FCF71DBBFFF7D1BE70B50446154676
:103EC0004618B44205D014F8010B2946FFF7E4FF69
:103ED000F7E700232B6770BD0120704708B5FFF797
:103EE00038FDBDE80840FCF71DBBFCF70DBBFFFF2C
:103EF0000248029A0C21FFF7E0BF00BFD241000048
:103F000000207047002070470020704700230B609E
:103F10004B606FF00B007047002303606FF00B00E5
:103F20007047002303606FF00C0070470B6C181A89
:103F300008647047704700207047FFFF13B50023E7
:103F40000A4A0B4C9A5C1A550133B3F50F7FF7D12F
:103F5000084909488DE81200A1F5005143F6F942DD
:103F60000B46FFF71DFB204602B010BDE4410000E8
:103F7000448BFF1F44B3FF1F20440000617070009A
:103F800000151915000100006487FF1F12000000D2
:103F9000000200008E87FF1F4300000000030000A6
:103FA000E887FF1F00000000010309047687FF1F58
:103FB0000000000002030904D287FF1F0000000078
:103FC00003030904EC87FF1F00000000000000004D
:103FD0000000000000000000050E08090D0C060797
:103FE0000F04001303931A9217C585848687C4FFB4
:103FF0004008FE4340A004404408FE4344A004405F
:104000000018FE4300C004403000FE4330900440DE
:104010003400FE43349004401C18FE431CC004408E
:104020001018FE4310C004400818FE4308C00440A6
:104030000C18FE430CC004400C10FE430CB00440AE
:104040001010FE4310B004401810FE4318B0044096
:104050001C10FE431CB004401410FE4314B0044076
:104060000418FE4304C004400010FE4300B00440A6
:104070000008FE4300A004400408FE4304A00440DE
:104080000C08FE430CA004400808FE4308A00440AE
:104090001418FE4314C004401818FE4318C004400E
:1040A0000410FE4304B004400810FE4308B004406E
:1040B0001400FE43149004404C08FE434CA00440FE
:1040C0000420FE4304D004402410FE4324B00440E6
:1040D0002010FE4320B004402810FE4328B00440C6
:1040E0002C10FE432CB004400020FE4300D00440BE
:1040F0004808FE4348A004401000FE4310900440CE
:104100006FF07F030370037813F0800FFBD07047CC
:1041100000547269656420746F20657865637574F6
:10412000652061206E756C6C20746F6B656E0A0083
:104130004F7574206F662064696374696F6E617275
:10414000792073706163650A00436F6E64697469F6
:104150006F6E616C73206E6F74207061697265643C
:104160000A00556E646566696E656420776F7264D7
:1041700020656E636F756E74657265640A004361D5
:104180006E27742066696E64202700270A00206964
:10419000736E277420756E697175650A0043204639
:1041A0006F72746820323030352E2020436F707962
:1041B00072696768742028632920313939372D32B4
:1041C000303035206279204669726D576F726B739B
:1041D0000A004E6F2066696C6520492F4F0A00FF68
:1041E000AF004800EA3C00003C0200000F00000065
:1041F000100000000000000000000000349A595533
:104200000F000000349A5955000000000000000023
:10421000C89C5955EC9F59550000000008A05755FF
:10422000FA195855F4985955FEFF000008A0595541
:10423000B89A5955F4985955000000000000000044
:10424000C89C5955F89F5955E01B0508D89C5955ED
:10425000D89C59550000000000000000FFFFFFFF40
:10426000FFFFFFFFFFFFFFFF000000000000000056
:10427000E89F5955882C0000EA3C0000000000002F
:1042800000000000570000000000000000000000D7
:10429000000000000000000000000000A40C00006E
:1042A0000000000000000000000000007E3600005A
:1042B000C3000000C300C3000000000000000000B5
:1042C00000000000000000000000000000000000EE
:1042D00000002A13000000000000000000000000A1
:1042E00000000000000000000000000000000000CE
:1042F0000000000000000000000C00004F1500004E
:104300000000000000000000000000004D00000060
:1043100000000000000C0000000C0000AB0F0000CB
:104320000000000000000000271A0000000000004C
:104330007E36000000000000000C000000000000BD
:1043400098330000369A595507000000000000001D
:104350004F00000008000000C61D0000851D000081
:10436000FFFFFFFF000C0000000000000000000045
:104370004B2A0000000000000000000000000000C8
:10438000E6220000AE230000000000000000000054
:10439000000000000000000000000000000000001D
:1043A0000000000000000000D12B0000B52D00002F
:1043B000000000000100000068031F08000000006A
:1043C000FFFFFFFF00000000FFFFFFFF00000000F5
:1043D000FFFFFFFFC72F0000000C0000000C0000D3
:1043E00000000000000000000000000000000000CD
:1043F00000000000000C00000000000000000000B1
:1044000000000000000000000000000000000000AC
:104410000D000000000000000060064000000000E9
:104420000000CB00CF00D300D700DA00DD00E000B1
:10443000E500E900ED00F200F700FC0000010501D5
:1044400009010E01130118011D0121012501290196
:104450002D013101350139013D014201450148017C
:104460004B014F01530157015B015F01630167017C
:104470006B016F01730177017B017F01830189016A
:104480008C019001940198019E01A101A501A9014F
:10449000AD01B301B901BF01C301C801CE01D30110
:1044A000D901DE01E501EA01ED01F001F601FC01AF
:1044B000020207020D02140218021D022202260245
:1044C0002B02300235023A023F02490251025902E0
:1044D0005F0266026B02700277027A027F02830239
:1044E00088028D02950298029B02A102A402AB02EF
:1044F000B002B702BD02C302CA02D202DA02E1026E
:10450000E702EE02F502FB02010305030B031003B1
:1045100016031D03240329032F03340339033E0329
:1045200044034A03500355035B035F0364036803BA
:104530006C037003740378037C037F038303890394
:104540008E03940398039C03A203A803AD03B40352
:10455000BA03BF03C503CE03D603DC03E203E803BB
:10456000EE03F703FC03010406040A041004170415
:104570001C04220428042E0435043C0446044E0482
:1045800056045F0464046B046F0476047E048404A0
:104590008B04930497049B049F04A704B004666FE4
:1045A000727468050000C5000000000000696E76A6
:1045B00065727406C3000100616E6403CB000200E3
:1045C000006F7202CF000300786F7203D300040003
:1045D0002B01D70005002D01DA0006002A01DD00BD
:1045E0000700736869667405E00008003E3E6103D9
:1045F000E500090064757003E9000A000064726F49
:104600007004ED000B00007377617004F2000C0081
:10461000006F76657204F7000D006E697003FC0090
:104620000E00007475636B0400010F00726F740359
:1046300005011000002D726F740409011100007053
:1046400069636B040E01120000726F6C6C0413013D
:104650001300003F6475700418011400003E7202DC
:104660001D01150000723E02210116000072400279
:1046700025011700323E72032901180032723E03F1
:104680002D0119003272400331011A0069702103B3
:1046900035011B006970400339011C0064657074AA
:1046A00068053D011D003C0142011E003D01450120
:1046B0001F003E014801200000303C024B01210058
:1046C00000303D024F01220000303E025301230022
:1046D00000753C025701240000312B025B012500CC
:1046E00000322B025F01260000322D0263012700F9
:1046F000756D2A0367012800006D2A026B012900ED
:104700006D2A2F036F012A0000322F0273012B0044
:104710006D61780377012C006D696E037B012D00BC
:10472000616273037F012E00006E65676174650628
:1047300083012F00400189013000006340028C0199
:1047400031000077400290013200006C4002940179
:10475000330000746F6B656E4006980134002101D0
:104760009E01350000632102A1013600007721027D
:10477000A5013700006C2102A901380000746F6B9D
:10478000656E2106AD0139006272616E63682107B2
:10479000B3013A006272616E63684007B9013B0081
:1047A000002B2102BF013C00636D6F766505C301DC
:1047B0003D0000636D6F76653E06C8013E000066F1
:1047C000696C6C04CE013F00636F6D7061726507A8
:1047D000D3014000636F756E7405D90141002D74DB
:1047E0007261696C696E6709DE01420063656C6C19
:1047F0002B05E50143006901EA0144006A01ED016E
:104800004500006272616E636806F00146003F6217
:1048100072616E636807F601470000756E6E65731E
:104820007406FC01480000657869740402024900BE
:10483000657865637574650707024A0000626568FC
:104840006176696F72080D024B006B657903140283
:104850004C00006B65793F0418024D0000656D69DE
:1048600074041D024E000063720222024F000074A5
:1048700079706504260250003E626F6479052B0250
:104880005100616C6C6F7405300252007666696E7F
:104890006405350253002466696E64053A025400CB
:1048A0007365617263682D776F72646C6973740FDE
:1048B0003F025500002463616E6F6E6963616C0A8C
:1048C00049025600007379732D6163636570740A41
:1048D0005102570000616363657074065902580005
:1048E000696E74657270726574095F025900616265
:1048F0006F72740566025A007468726F77056B02F6
:104900005B000066696E69736865640870025C002C
:10491000300177025D000068657265047A025E000E
:10492000746962037F025F00002F7469620483026E
:1049300060007061727365058802610000706172C9
:1049400073652D776F72640A8D0262002C019502E7
:1049500063003B81980264003A6E6F6E616D65077B
:104960009B0265003A01A102660000636F6E7374DA
:10497000616E7408A4026700007573657204AB026F
:104980006800007661726961626C6508B002690056
:104990000063726561746506B7026A002468656128
:1049A00064657207BD026B0000636F6C6F6E2D63F0
:1049B0006608C3026C00636F6E7374616E742D635E
:1049C000660BCA026D00006E6E7661726961626C80
:1049D000650AD2026E006372656174652D636609B3
:1049E000DA026F002463726561746507E10270008A
:1049F000757365722D73697A6509E7027100696DD7
:104A00006D65646961746509EE027200002B6C6566
:104A100076656C06F5027300002D6C6576656C0694
:104A2000FB0274002827290301037500002863682E
:104A30006172290605037600286C697429050B0349
:104A400077000028776C6974290610037800787461
:104A50006C69746572616C091603790000636F6D8F
:104A600070696C652C081D037A00006475702E0453
:104A700024037B00003F6C656176650629037C009A
:104A80006C65617665052F037D00283F646F2905FD
:104A900034037E000028646F290439037F00002856
:104AA0006C6F6F7029063E038000282B6C6F6F704F
:104AB0002907440381000028646F657329064A03AF
:104AC000820000282E22290450038300636F6D703A
:104AD000696C650755038400627965035B03850093
:104AE000006C6F7365045F0386007370400364039A
:104AF00087007370210368038800727040036C03A1
:104B000089007270210370038A007570400374037A
:104B10008B007570210378038C002F017C038D00BE
:104B20006D6F64037F038E0000782A2F6D6F64061B
:104B300083038F00002F6D6F640489039000646EFF
:104B40006567617465078E03910000642D0294030C
:104B5000920000642B029803930000756D2F6D6F17
:104B600064069C03940000736D2F72656D06A203AA
:104B70009500646967697405A803960000246E7542
:104B80006D6265723F08AD0397003E6E756D62659C
:104B90007207B4039800006869646504BA03990059
:104BA0000072657665616C06BF039A0000696E74D9
:104BB00065726163746976653F0CC5039B006D6F18
:104BC00072652D696E7075743F0BCE039C00006F8B
:104BD000726967696E06D6039D0000756E75736510
:104BE0006406DC039E00002F746F6B656E06E203A3
:104BF0009F002F6272616E636807E803A000006D7A
:104C000061787072696D69746976650CEE03A10054
:104C100063656C6C7305F703A2006363616C6C05DC
:104C2000FC03A3006163616C6C050104A4000062D5
:104C30006C020604A50000736561726368060A04CD
:104C4000A60000616C6C6F63617465081004A700B6
:104C50000066726565041704A80000726573697ABE
:104C600065061C04A9003E72656C62697407220423
:104C7000AA0000666C6F61743F862804AB0067650C
:104C8000742D6C6F63616C092E04AC007365742D18
:104C90006C6F63616C093504AD00616C6C6F6361AE
:104CA00074652D6C6F63616C730F3C04AE006672AB
:104CB00065652D6C6F63616C730B4604AF00006C0F
:104CC0006F63616C2D6E616D650A4E04B000646F98
:104CD0002D6C6F63616C2D6E616D650D5604B100B6
:104CE0000073617665045F04B200726561642D6CC7
:104CF000696E65096404B300722F6F036B04B4001E
:104D00006F70656E2D66696C65096F04B500006390
:104D10006C6F73652D66696C650A7604B600007465
:104D20006F2D72616D067E04B700726561642D6639
:104D3000696C65098404B8000077726974652D6632
:104D4000696C650A8B04B900772F6F039304BA006E
:104D5000722F77039704BB0062696E039B04BC004B
:104D60006372656174652D66696C650B9F04BD0097
:104D70000073706C69742D737472696E670CA7048C
:104D8000BE00283A2903B004C000BF00000000287C
:104D9000636F6E7374616E74290AB404C000C0003E
:104DA000000000287661726961626C65290ABE04A0
:104DB000C000C100000000286372656174652908A5
:104DC000C804C000C200000000287573657229067F
:104DD000D104C000C300000028646566657229071D
:104DE000D904C000C40000000028766F63616275BA
:104DF0006C617279290CE104C000C5000000002834
:104E0000636F64652906EC04C000C60000002876C4
:104E1000616C75652907F404C000C70000002375A4
:104E200073657205FC04C30004003E696E0303054C
:104E3000C30008000062617365040805C3000C002C
:104E4000626C6B030E05C3001000002374696204DA
:104E50001305C30014000027746962041905C30018
:104E6000180023736F75726365071F05C3001C006C
:104E700027736F75726365072605C300200073747E
:104E8000617465052D05C300240064656C696D6956
:104E9000746572093305C3002800277370033B054E
:104EA000C3002C00277270034005C3003000276642
:104EB00070034505C3003400276F726967696E0788
:104EC0004A05C3003800006470025105C3003C006D
:104ED00000276C696D6974065605C3004000002701
:104EE00072616D6374065D05C30044000027726142
:104EF0006D746F6B656E730A6405C300480000270C
:104F0000636F6D70627566086D05C3004C00276C99
:104F10006F63616C73077505C300500000736176A1
:104F200065642D6470087C05C30054007361766568
:104F3000642D6C696D69740B8405C300580073702F
:104F400030038D05C3005C00727030039205C3000E
:104F50006000757030039705C30064002772737397
:104F6000617665079C05C30068002772736D6172E6
:104F70006B07A305C3006C0000236F757404AA05BA
:104F8000C3007000236C696E6505B005C300740032
:104F900064706C03B605C30078007761726E696E49
:104FA0006707BB05C3007C00006361707304C20522
:104FB000C3008000765F6572726E6F07C805C3001C
:104FC000840023706C6163657307CF05C30088009C
:104FD00068616E646C657207D605C3008C0000764C
:104FE0006F632D6C696E6B08DD05C3009000006C6B
:104FF00061737404E505C30094000027696E74654D
:1050000072707265740AEB05C300980027717569A8
:105010007405F405C3009C00276163636570740721
:10502000FA05C300A0007468697364656607010629
:10503000C300A400636F6D706C6576656C0908062B
:10504000C300A8000023696E73041006C300AC00FF
:10505000006C6F636E756D061606C300B000277393
:105060007973707472071D06C300B40000626F7517
:105070006E64617279082406C300B8003C6970034D
:105080002C06C300BC0069703E033106C300C0009B
:10509000636E74033606C300C4000027646562753E
:1050A00067063B06C300C80063757272656E7407BD
:1050B0004206C300CC00636F6E74657874074906BE
:1050C000C300D0005D0066616C7365055006C000CA
:1050D000000000000074727565045706C000FFFFF1
:1050E000FFFF5B815E06BF005706330535004800B1
:1050F0005D016306BF005E063305350048006C693C
:10510000746572616C876A06BF000A005E003A002F
:105110005E003B000D001F00470012008400780075
:105120005E003A00A00052004600080084007700AC
:10513000630048000032647570047406BF000D00FF
:105140000D0048003273776170058E06BF001000B5
:1051500015001000160048003264726F7005960644
:10516000BF000B000B00480000736F75726365068B
:10517000A006BF002D053000260530004800007352
:1051800065742D736F757263650AA906BF002605E5
:1051900035002D05350048000027736F7572636573
:1051A0002D69640AB606C3001001736F75726365DA
:1051B0002D696409C306BF00C306300048000073B0
:1051C0006176652D696E7075740ACB06BF00A906FD
:1051D000CB060805300013053000770005000000FD
:1051E0004800726573746F72652D696E7075740D09
:1051F000D606BF000B001305350008053500C306B1
:105200003500B606570648007365742D696E7075D3
:105210007409E906BF005D005D007700050000002D
:10522000E9060B0048002F737472696E6707FA066F
:10523000BF000F000600110005000C0048000077B9
:105240006865726531060807BF00A90683000A4534
:1052500072726F722061743A20000D0008053000F0
:105260005000830004207C2020000805300008073F
:1052700050004F004800002E6E6F742D666F756EE3
:10528000640A1407BF004F005000830002203F0053
:105290004F001407480024646F2D756E64656669BD
:1052A0006E65640D3207BF003207330530004700DA
:1052B0000A0084008600460006004F005A0048009D
:1052C000646570034307BF001D007B000B004F00A7
:1052D000480000636F6D70696C652D776F72640CA8
:1052E0005307BF0054000A0047001A00210033058D
:1052F00030000200470008007A00460004004A001F
:1053000046003C000B008E069700470030009606D2
:10531000A006BB053000470012000B00330530002B
:1053200047000400740646001000330530004700B3
:1053300008000C0074067406460004004307480089
:105340000028696E746572707265740A6107BF0027
:1053500062000A004700080061074600F4FFA0064B
:105360004800003F626C6F636B2D76616C69640C62
:105370009707BF005706480000726566696C6C06A7
:10538000A907BF0013053000470010007700010097
:10539000000013053C00A9074900CB067700FFFF7A
:1053A000FFFF1F004700060057064900A9060B0033
:1053B000CB06470056006000CB06B30047001C0038
:1053C00083001472656164206572726F7220696E69
:1053D00020726566696C6C005A000D0060001F0049
:1053E0004700240083001B6C696E6520746F6F207A
:1053F0006C6F6E6720696E20696E707574206669C7
:105400006C6500005A0046001400600058000A0055
:10541000470008005E06460004009C000C002605BC
:1054200035005D00080535004800003F3F63720409
:10543000B107BF00B0053000470004004F0048002E
:105440006361746368050908BF0087001500DD0506
:10545000300015008900DD0535004A005D001600AA
:10546000DD05350016000B0048000073746174758B
:1054700073061408C40014010070726F6D70740616
:105480002A08BF009B00470020002A08330530008F
:1054900047000E00830003205D20000046000A0044
:1054A0008300036F6B2000004800636C6561720528
:1054B0003108BF009205300088004800002E657258
:1054C000726F72064908C400180127657869742D47
:1054D000696E7465726163743F0F5308C3001C01E9
:1054E00000696E746572616374085E08BF005F00D6
:1054F00060005D00FA0663061D00210047001A00E7
:1055000083000F537461636B20556E646572666C23
:105510006F7700004F0049083108B10747001C00B1
:105520007500970714080908140047000600630671
:1055300053085E0830004700C0FF57065E0835007C
:1055400048000071756974046608BF005D001006AC
:105550003500970530008A00660885004800696EAE
:10556000746572707265742D6C696E65730F950841
:10557000BF00B1074700080097074600F6FF480044
:10558000006576616C7561746508A808BF00D60671
:105590001800180018007700FFFFFFFFFA067500DB
:1055A00097071408190019001900E9065B005B0051
:1055B000480000696E636C7564652D66696C650CE6
:1055C000B608BF006000A7005B00D60618001800F0
:1055D000180060001000FA067500A80814080A00F8
:1055E000470004001407CB06B6000B00A9060B0009
:1055F000A8000B00190019001900E9065B005B0008
:10560000480000696E636C7564656408D108BF006A
:10561000B400B5005B00D1084800696E636C756426
:10562000696E6709F708BF006200F7084800006666
:105630006C020309BF0003094800666C6F616405D2
:105640000A09BF0003094800686578031109BF0013
:10565000780010000E0535004800646563696D61CF
:105660006C071709BF0078000A000E0535004800D6
:1056700000632C022209BF005E0078000100520086
:10568000360048005C812B09BF00A90608053500DB
:105690000B0048000063686172043409BF006200B7
:1056A0000B0031004800005B636861725D863E0953
:1056B000BF003E0984007600630048002881480945
:1056C000BF007600290000006100A0064800002EFF
:1056D00028825009BF0076002900000061005000B8
:1056E0004800736166652D70617273652D776F7206
:1056F000640F5A09BF0062000A0022005B004800E4
:105700000024646566696E6564086A09BF006A09F9
:105710005400480027017609BF00620054002200AF
:105720005B0048005B275D837C09BF007C09790032
:1057300048005B636F6D70696C655D898509BF00AA
:105740007C097A004800646F65733E858F09BF004D
:10575000840082004800003C7265736F6C766508B7
:105760009709BF005E0006005E003A00A0005200EC
:1057700048003E6D61726B05A109BF005E000A0022
:10578000A1094800003E7265736F6C766508AD092B
:10579000BF005E000D0006000C003A0048003C6DA2
:1057A00061726B05B809BF005E004800006966823F
:1057B000C309BF00730084004700AD094800616859
:1057C00065616485C909BF00730084004600AD09A6
:1057D0004800626567696E85D309BF007300C3091D
:1057E0004800007468656E84DD09BF00B809740064
:1057F0004800756E74696C85E509BF008400470038
:10580000A10974004800616761696E85ED09BF00F8
:1058100084004600A1097400480063732D726F6C08
:105820006C07F709BF001300480063732D706963AC
:105830006B07020ABF0012004800627574830A0AEF
:10584000BF0078000100020A480079657483100ADD
:10585000BF005D000A0A480000646F82180ABF009A
:10586000730084007F00AD0948003F646F831F0A06
:10587000BF00730084007E00AD094800006C6F6FAC
:105880007084280ABF0084008000180AA000050068
:10589000A109B809740048002B6C6F6F7085320A3B
:1058A000BF0084008100180AA0000500A109B80902
:1058B000740048007768696C6585400ABF00C909B3
:1058C000100A480000656C7365844E0ABF00D30956
:1058D000100AE50948000072657065617486560A11
:1058E000BF00F709E509480000787768657265062A
:1058F000600ABF00480000706F7374706F6E658837
:10590000690ABF00620054000A002200470010002C
:105910000B00CE0FA0068400860046000E0021007A
:1059200047000600840084007A004800003C3E02E4
:10593000710ABF001F00220048000063656C6C0400
:10594000890AC000040000003F5C6D617463680751
:10595000910ABF00890A4700040034094800333225
:105960005C83990ABF00910A78000400990A4800F4
:1059700031365C83A20ABF00910A78000200990ABE
:105980004800005C74313684AB0ABF009F00780089
:105990000200990A4800005C74333284B50ABF00E3
:1059A0009F0078000400990A4800002F6302BF0A94
:1059B000C00001000000002F7702C80AC0000200EA
:1059C0000000002F6C02CE0AC0000400000000633B
:1059D00061312B04D40ABF002500480000776131F3
:1059E0002B04DB0ABF0026004800006C61312B0449
:1059F000E20ABF00D40A050048002F632A03E90A1F
:105A0000BF0048002F772A03F00ABF000A000500F4
:105A100048002F6C2A03F50ABF00A2004800006F5F
:105A20006B02FC0ABF004800747269676765728781
:105A3000020BBF005D005D00180019000B000B0099
:105A4000480000782E02090BBF000A007800000011
:105A5000780000004F004800002F6E02140BBF00BA
:105A600078000100A2004800006E61312B041F0B7A
:105A7000BF00430048006E612B03280BBF00A2004B
:105A8000050048000023616C69676E062E0BC0009C
:105A90000200000000312D02370BBF00780001002A
:105AA0000600480000322A023D0BBF0078000200C9
:105AB00007004800326F76657205450BBF0078001D
:105AC0000300120078000300120048000032400278
:105AD0004E0BBF000A001F0B050030000C00300009
:105AE000480000322102590BBF000C000D003500A8
:105AF0001F0B050035004800003E3D02640BBF004F
:105B00001E0022004800753C3D036F0BBF008E064F
:105B1000240011001F000300480000753E02760BB0
:105B2000BF00760B22004800753E3D03800BBF008E
:105B3000240022004800003C3D02870BBF002000EB
:105B400022004800303C3E038E0BBF0022002200A2
:105B50004800303C3D03950BBF000A0022000C00BA
:105B6000210003004800303E3D039C0BBF00210094
:105B70002200480000287382A60BBF00500948008D
:105B800070616403AD0BBF005E0078006400050027
:105B90004800737061636505B30BBF00A5004E003C
:105BA00048000073706163657306BD0BBF005D0044
:105BB0007E000800BD0B8000FCFF480000666D2FD2
:105BC0006D6F6406C60BBF008E06040021004700FF
:105BD00022000A00150095000D00470010003D0B43
:105BE0000C00160005000C004600060016000B0015
:105BF0004900950048002A2F6D6F6405D30BBF0044
:105C0000150029001600D30B4800002A2F02EF0BC5
:105C1000BF00EF0B0E004800006E6F6F7004F80BB2
:105C2000BF004800616C69676E656407000CBF00C7
:105C30007800010005007800FEFF02004800616C5A
:105C400069676E05070CBF005E005E00070C0C0064
:105C5000060052004800006C616C69676E6564085C
:105C6000130CBF007800030005007800FCFF020061
:105C70004800006C616C69676E06210CBF005E0015
:105C80005E00210C0C000600520048006572617332
:105C900065052E0CBF005D003F0048006F6666037F
:105CA0003A0CBF0057060C0035004800006F6E022A
:105CB000410CBF005E060C003500480000756D61A8
:105CC0007804490CBF008E062400470004000C0035
:105CD0000B0048000077697468696E06520CBF00BB
:105CE0000D0006001500060016002400480062653D
:105CF000747765656E075F0CBF0025005F0C480078
:105D0000007072696D69746976653F0A6C0CBF003A
:105D100078000100A1005F0C48006F6374616C059E
:105D2000770CBF00780008000E05350048000062BF
:105D3000696E61727906810CBF00780002000E0561
:105D400035004800007461312B048C0CBF009F00AB
:105D50000500480074612B03960CBF009F000700EC
:105D6000050048002F6C696E6B059D0CC000020099
:105D700000003E6C696E6B05A60CBF009F0006001C
:105D80004800003E666C61677306AD0CBF00AD0C49
:105D90003D0B480000696D6D6564696174653F0A7B
:105DA000B60CBF00B60C310078008000020048003D
:105DB000003E6E616D652406C10CBF00B60C0A0082
:105DC000310078003F0002000F0006000C00480080
:105DD0002E6E616D6505CD0CBF00CD0C5000BD0B66
:105DE00048006C61737461636607DC0CBF00EB05EF
:105DF00034004800626F64793E05E60CBF009F00E6
:105E000006004800006C736869667406EE0CBF00FB
:105E1000080048000072736869667406F70CBF00DA
:105E20002F0008004800003C3C02FF0CBF000800A7
:105E30004800003E3E02060DBF002F00080048004B
:105E4000636640030C0DBF00320048006366210307
:105E5000130DBF0037004800756E756D4005190DB4
:105E6000BF0032004800003E757365722306200DA6
:105E7000BF005100200D48003E7573657205280D66
:105E8000BF00200D8B000500480000277573657268
:105E90002306300DBF007C09280D4800776F72641F
:105EA0002D74797065093A0DBF000A00770C470020
:105EB0000A000B007800FFFF4900130D0A00770C61
:105EC000470008000B007800FFFF48000075616C78
:105ED0006C6F6306440DBF00030530000C00030522
:105EE0003C0048006E75736572055B0DBF001F0BAB
:105EF0005B0D68004800637261736805660D000001
:105F000017009F00060034000A0075000D021F00F4
:105F10004700060046000400DC0C48006465666526
:105F200072056F0DBF006A00E1045E00EE0C3700E1
:105F30005E001F0B5B0D6300300D75006F0D3900A7
:105F40004800646566787805820DC4002001000071
:105F500000746F6B656E2C06950DBF005E009F0090
:105F6000520039004800006E21029D0DBF0035002F
:105F700048006C696E6B4005A60DBF0034004800F8
:105F80006C696E6B2105AD0DBF00390048006C696E
:105F90006E6B2C05B40DBF009D0D48006E6F6E2D0D
:105FA0006E756C6C3F09BB0DBF000A009D00890A2D
:105FB0000A002200470004000E0048002C756E7590
:105FC0006D05C40DBF00030530005E003A00A0005F
:105FD000520003053C00480076616C756505D20DE2
:105FE000BF006A00FC045E00EE0C190D03053000D2
:105FF0001F0BD20D8B0005003500480069737661D8
:106000006C756507E00DC70024010028746F290432
:10601000F30DBF000A0051000C00130D0A00FC0430
:106020001F0047000A000B00300D350049000A0030
:10603000E1041F0047000A000B00300D3900490041
:106040000A00D9041F0047000A000B00300D35007C
:1060500049000A00EC041F0047000A000B00300D45
:10606000390049000B003500480000746F82F90DBB
:10607000BF003305300047000C0085098400F90D8E
:10608000460006007C09F90D4800006865616465FA
:106090007206280EBF006A096B00480064656669D5
:1060A0006E6974696F6E730B3A0EBF005006340050
:1060B000490639004800657869743F05450EC400FB
:1060C0002801000000626F756E6473064F0EBF00FA
:1060D0000D0005000C004800002E2E02570EBF00D8
:1060E0000A0030007800000078000000280B48000B
:1060F00000646F2D646566696E65640A5F0EBF009B
:1061000033053000470014002300470008004A0010
:10611000460004009D0D460006000B004A004800A2
:10612000007072696E7461626C653F0A6F0EBF0029
:10613000A50078007F005F0C4800636F6E74726F7B
:106140006C87870EBF006A090B003100A5003D0B6C
:106150000200330530004700040074064800006D5B
:106160006F766504920EBF0011008E062400470072
:106170000A0010003E004600060010003D004800E6
:10618000706C61636505A30EBF008E0636008E0637
:10619000050025005D000C00360025000C00A30E54
:1061A0004800007061636B04B40EBF000A00150064
:1061B000B40E16004800657874726163742D7374B0
:1061C000720BC50EBF0041008E0605002500070CAE
:1061D0001100480000222C02D20EBF000F005E000A
:1061E000B40E26005200130C4800736B6970737470
:1061F0007207DD0EBF0016001C00D20E10001B003F
:10620000100015004800002822732904EA0EBF0080
:10621000EA0E0B003D0B480028222903F70EBF00B1
:10622000EA0E480000736C69746572616C88FF0E39
:10623000BF008400FF0EDD0E480000732282080FAD
:10624000BF007600220000006100330530004700E7
:106250000400080F4800002863222904100FBF0023
:10626000EA0E0B00480063736C69746572616C8997
:106270001F0FBF0084001F0FDD0E48000063228245
:10628000290FBF0076002200000061008E06050085
:106290005D000C0036003305300047000800290F70
:1062A000460004000B004800002C2202310FBF0002
:1062B0007600220000006100DD0E4800002E2282E0
:1062C000470FBF003305300047000C0084008300F7
:1062D000470F46000C0076002200000061005000CD
:1062E00048002761626F72742407510FC3002C01AC
:1062F0000000002861626F7274222908660FBF00D7
:1063000047001600EA0E0B003D0B660F35007800C3
:10631000FEFF5B0046000600EA0EA0064800006192
:10632000626F727422866F0FBF0084006F0F470F79
:1063300048006C303D03840FBF0022004800006518
:1063400072726F722D6F75747075740C8C0FC4003F
:106350003001000000726573746F72652D6F757483
:106360007075740E970FC400340100000028776820
:1063700065726506A30FBF009B004700360033051A
:1063800030004700140083000A436F6D70696C6928
:106390006E672000460016008300104C6174657320
:1063A0007420776F7264207761732000E60CDC0C38
:1063B0004F004800776865726505AB0FC40038016F
:1063C0000000003F737461636B06CE0FBF0087004F
:1063D000920530000C00240047002400970F830032
:1063E00010537461636B20556E646572666C6F77D1
:1063F0002000CE0FA30F9205300088005A008700BE
:106400009205300078009001060024006F0F0F53B2
:106410007461636B204F766572666C6F7720000045
:10642000480063737003D60FC3003C0100000021D5
:10643000637370040410BF00870004103500480027
:10644000003F637370040B10BF008700041030001E
:10645000890A47001C00970F83000E537461636B19
:10646000204368616E6765642000CE0FA30F5A0059
:106470004800002769021410BF0076090A002200B4
:10648000470008000B0032075A004800007365748B
:10649000616C696173082C10BF000C009D0D6300D6
:1064A000720082000A0034000C00960C30006F0E5F
:1064B0004800616C696173053C10BF006A00990077
:1064C0002C109A003C1048000033322D626974860B
:1064D0004D10BF0048000031362D62697486591096
:1064E000BF00780001006F0F124E6F7420612031E1
:1064F000362062697420666F7274680048006C64AC
:10650000726F7085601042100B00FFFFFFFF006C80
:1065100064757084731042100A00FFFFFFFF006C67
:106520002B827B1042100500FFFFFFFF756C2A8352
:10653000821042100700FFFFFFFF6C2B21838910A0
:1065400042103C00FFFFFFFF006C6E6F76657286A5
:10655000901042100D00FFFFFFFF006E6C6F76651C
:106560007286991042100D00FFFFFFFF006E6C73E2
:1065700077617086A21042100C00FFFFFFFF006CD5
:106580006E7377617086AB1042100C00FFFFFFFF47
:106590006C7377617085B41042100C00FFFFFFFF31
:1065A000006C3D82BC1042101F00FFFFFFFF006C1B
:1065B0003C82C31042101E00FFFFFFFF6C3E3D8374
:1065C000CA1042106F0BFFFFFFFF006C6C6974650F
:1065D00072616C88D1104210740601000000006CDA
:1065E000616E6484DB1042100200FFFFFFFF6C6EDF
:1065F000656761746587E31042102F00FFFFFFFF9E
:10660000006C2C82EC1042106300FFFFFFFF6C72E5
:106610003E83F31042101600FFFFFFFF6C3E7283B3
:10662000FA1042101500FFFFFFFF006C2D3E6E8434
:106630000111BF00480000772D3E6C840911BF0096
:10664000480000732D3E6C040F11BF000A00770054
:1066500000800000020047000E0077000000FFFFEE
:10666000030046000A007700FFFF00000200480018
:106670006C7661726961626C6589151142106900FE
:10668000FFFFFFFF6C636F6E7374616E74892E1170
:1066900042106700FFFFFFFF006E2D3E77043811A8
:1066A000BF007700FFFF000002004800006E2D3E93
:1066B0006C84401142100F1101000000733E64030E
:1066C0004A11BF000A0021004800753E64035111C1
:1066D000BF005D00480063612B8358114210050024
:1066E000FFFFFFFF77612B035E11BF00F50A050076
:1066F00048006C612B036511BF00FC0A05004800CF
:1067000000772C026C11BF005E00CE0A52003700E9
:1067100048003C7740037311BF0032001511480058
:10672000006973827C114210280E01000000686C21
:1067300064038311C3004001000000686F6C6404AF
:106740008A11BF007800FFFF8A113C008A113000D7
:1067500036004800003C23029111BF00B30B8A11A0
:106760003500480000233E029D11BF00A0068A119B
:106770003000B30B0D0006004800007369676E041B
:10678000A511BF00210047000A0076002D0000007F
:1067900091114800006D752F6D6F6406B111BF0037
:1067A00015005D001700940016000C001500940001
:1067B000160048002301BF11BF000E053000BF11B5
:1067C00010000A007800090020004700140078003B
:1067D0000A000600760061000000050046000A007D
:1067E00076003000000005009111480064303D0340
:1067F000CC11BF0003002200480000237302E911FE
:10680000BF00CC118E06E9114700F8FF48000028B0
:10681000752E2904F011BF0058119D11F011A5111A
:10682000480000752E02FB11BF00FB115000BD0B8C
:106830004800752E72030412BF001500FB111600EC
:106840000D000600C60B50004800282E29030C122C
:10685000BF000A002E0058119D11F0111000B11157
:10686000A511480000732E021812BF001812500024
:10687000BD0B48002E012512BF000E053000780028
:106880000A001F00470008002512460004000412F9
:106890004800002E72022C12BF00150018121600BC
:1068A0000D000600C60B50004800006C2E823C1202
:1068B00042102C12FFFFFFFF282E73034812BF0067
:1068C0001D005D007E0012001D00440006003D0B0F
:1068D00012002C128000F2FF4800002E73024F12AB
:1068E000BF00D60F1D00470008004F1246000C00E5
:1068F000830006456D7074792000480073686F77D7
:10690000737461636B096012BF0075004F127500EC
:106910002A08F90D48006E6F73686F7773746163AE
:106920006B0B7412BF007500000C75002A08F90D7E
:1069300048003F018212BF0030002C124800002E98
:1069400078028B12BF000E0530000C0017092C12C4
:106950000E05350048006E64756D70059212BF001B
:10696000570E7E000E00440030002C121F0B8100D9
:10697000F6FF48007764756D70059F12BF00570ED3
:106980007E001000440032002C12780002008100CA
:10699000F4FF48006364756D7005AE12BF00570EBA
:1069A0007E000C00440031002C128000F8FF4800EB
:1069B00023766F637305BE12C00010000000002331
:1069C0007468726561647308CC12C0000100000035
:1069D00000766F636162756C6172790AD512BF00CF
:1069E0006A005E00EE0C03053000D512A200D20D45
:1069F0008B000500D5125D007F000E009D000D008C
:106A00003900960C8000F6FF0B00E505AD0DBB0DBF
:106A1000E505B40D8200EE0C500639004800616EA9
:106A20006F746865722D6C696E6B3F0DDF12BF006D
:106A3000AD0DC40D4800003E746872656164730852
:106A40000713BF005100300D48003E766F632D6C78
:106A5000696E6B091113BF005100A00005004800CA
:106A600000766F633E041B13BF00480000726F6F17
:106A700074042413FB124401C30000616C736F049F
:106A80000000BF0050060A00960CCC1227009F00A1
:106A900007003E004800006F6E6C79043113BF00A0
:106AA000CC125D007F0010009D00500644009D0C3C
:106AB00039008000F4FF75002A135006CC123D0BFC
:106AC0009D0C39002A134800007365616C043F1364
:106AD000BF007C0951005006CC121F0B07003A0C76
:106AE0005006390048000070726576696F7573084A
:106AF0005813BF0050060A00960C0C00CC12270059
:106B00009F0007003D005006CC1227009F000700A1
:106B100005009D000C0039004800666F727468051E
:106B20006913BF00C3004800646566696E697469D3
:106B30006F6E730B8113BF00450E48006F72646562
:106B400072058B13BF00830009636F6E74657874E0
:106B50003A2000005006CC125D007F0014000A00AD
:106B60003400C40D47000400DC0C960C8000F0FFDC
:106B70000B0078000400C60B830009637572726510
:106B80006E743A20000049063400DC0C48000076A0
:106B90006F6373049213BF00E505071347000C00F1
:106BA0000A00DC0C1B134600F2FF48006C617267A0
:106BB00065737407BB13C1004801000000666F6C69
:106BC0006C6F7706CB13BF001113AD0DCB13B40D53
:106BD000480000616E6F746865723F08D313BF0090
:106BE000CB13AD0DC40D470012000A00AD0CAD0D66
:106BF000CB13B40D5E06460004005706480000683B
:106C0000696464656E062A13FB124C012A136470D2
:106C10002103F413BF005E000600520048006665C1
:106C20006E636505FA13C3005001000000747269B9
:106C30006D040314BF00D5125D007F001C008E069A
:106C4000AD0D8E06800B4700F8FF0E000D00B40D51
:106C5000A60C05008000E8FFA006480028666F72B9
:106C6000676574070A14BF00AD0C0A000314AD0D6C
:106C700024006F0F0B62656C6F772066656E63652D
:106C800000000A00E505AD0D8E06870B4700F8FFF2
:106C90000A00E505B40D0E000A009D00890A4700B0
:106CA0000E008E0611130A14AD0D4600ECFF0B000A
:106CB000FA13480000666F72676574062314BF00FC
:106CC0006A0949063000550022006F0F1943616EB2
:106CD00027742066696E6420776F726420746F2059
:106CE000666F726765740000231448003F636F6D20
:106CF00070054F14BF003305300022006F0F1143A1
:106D00006F6D70696C6174696F6E204F6E6C792065
:106D1000000048003F65786563056A14BF003305CD
:106D200030006F0F0F457865637574696F6E204F83
:106D30006E6C792000004800003F70616972730634
:106D40007E14BF0006006F0F18436F6E646974698C
:106D50006F6E616C73206E6F742070616972656410
:106D6000200048002F6E2A039114BF007800020013
:106D7000060D4800007265616404A514C00000009F
:106D80000000777269746505AE14C0000100000050
:106D9000006D6F6469667906B514C00002000000DA
:106DA0007265637572736587BD14BF00E60C7A0067
:106DB00048006E6F7483C51442100100FFFFFFFF8F
:106DC000636861727305CC14BF0048006368617228
:106DD0002B05D414BF002500480000756E6C6F6F42
:106DE0007006DA14BF00160016000B0016000B0028
:106DF00016000B0015004800626C616E6B05E21412
:106E0000BF00A5003F004800706175736505F01470
:106E1000C400540100003364726F7005F814BF00A1
:106E2000A0060B00480000707573682D686578082F
:106E3000FF14BF0016000E053000150015001709DD
:106E4000480000707573682D646563696D616C0C32
:106E50000915BF0016000E053000150015002209A7
:106E6000480000706F702D62617365081915BF00CE
:106E7000160016000E05350015004800002E6402AD
:106E80002715BF0019152C1227154800002E68027F
:106E90003115BF000915041227154800002E616244
:106EA0006F7274063915BF00660F30004100500044
:106EB000480000282E6572726F7229084315BF00C2
:106EC0000A007800FEFF1F00470008004315460037
:106ED0002C000A007800FFFF1F00470014000B0081
:106EE00083000741626F72746564000046000E0003
:106EF0008300064572726F72200031154F00480002
:106F0000286372034F15BF0078000D004E00480043
:106F1000007523027315BF005D00CC110B00480003
:106F2000752373037B15BF005D00F0110B00480053
:106F300075233E038315BF005D00A5114800006E58
:106F4000756C6C737472696E670A8B15C2000000F1
:106F5000246E756D626572079615BF009700470035
:106F60000A000B005706460004005E064800753212
:106F70002F039D15BF0078000100FF0C4800007230
:106F80006F756E642D757008AA15BF003D0B0F005C
:106F900005000C00010002004800616C6C6F632D5D
:106FA0006D656D09B515BF00A7005B004800006660
:106FB0007265652D6D656D08C315BF000B00A800D7
:106FC0005B00480000707572706F73653A88CD156C
:106FD0004210340901000000006865616465726C4C
:106FE0006573738AD8154210000CFFFFFFFF6865B8
:106FF000616465727387E3154210000CFFFFFFFFA9
:1070000028656D697405EC15BF00B00530000C00F3
:107010004E00B00535004800287479706505F415F8
:10702000BF00B005300011005000B0053500480029
:10703000757063030016BF00780020000100020095
:107040004800232D627566850B164210B30BFFFFB7
:10705000FFFF6C6F6E672D636F6D6D656E74730DE2
:107060001516C1005801000028812116BF0008052F
:10707000300076002900000061000E0005000805C0
:1070800030001F0021163000CB067800FFFF5D00A6
:107090006C0C22000300020047001000B107220020
:1070A0004700040049004600C6FF4800002F7573E2
:1070B000657223062616C00004000000627566662D
:1070C00065722D6C696E6B0B4B16C3005C01000082
:1070D0000075736572232C065516BF00030530003A
:1070E0000A0063000C0003053C008B00050048000B
:1070F0006D616B652D6275666665720B5D16BF000E
:107100005E00EE0C0C005D001F0B5D163500630089
:107110005516AD0DBB0D5516B40D480000616C6CD5
:107120006F632D6D656D340A6F16BF007800040023
:107130000500C31578000400B5154800646F2D6282
:107140007566666572098516BF000A00300D30004D
:1071500047000A00300D300046001C000A004B16A4
:10716000050030000A0085160A0010003A0C0A00DB
:107170001000300D35004800286275666665723A69
:1071800029099416BF006F006F16820094164800FC
:107190006275666665723A07B216BF003A0EB2169D
:1071A0004800003E6275666665722D6C696E6B0CF8
:1071B000BD16BF0051004B160500780001002E0BD4
:1071C000480000636C6561722D6275666665723A8F
:1071D000730EC916BF0055160713470010000A00AA
:1071E0005100300D410CC9164600EEFF4800002E3C
:1071F0006275666665727308DA16BF005516071366
:1072000047001A000A00DC0C0A0051004B1605006A
:1072100030002C124F00C9164600E4FF4800003F22
:107220005C82ED16BF0022004700040034094800CC
:10723000005C3F820217BF00620054000A00470052
:1072400008000E00460006000E000E00021748005F
:10725000005B656C73655D860B17BF0078000100ED
:1072600062000A004700940056008E06FF0E045B81
:1072700069665D004000220015008E06FF0E075B68
:1072800069666465665D0000400022001600030028
:1072900015008E06FF0E085B69666E6465665D000C
:1072A000400022001600030047000A00A006250047
:1072B000460044008E06FF0E065B656C73655D003C
:1072C0004000220047001200A0063D0B0A004700C4
:1072D0000400250046001600FF0E065B7468656E0C
:1072E0005D0040002200470004003D0B1400220016
:1072F000470004004900460068FFA006B1072200CD
:1073000047005EFF0B004800005B69665D841D1747
:10731000BF002200470004001D174800005B74688E
:10732000656E5D867817BF0048005B6966646566B8
:107330005D878317BF0076090E000A002200470010
:1073400004000E0078174800005B69666E6465668D
:107350005D888A17BF0076090E0022000A004700E8
:1073600004000E00781748000063617365849A1763
:10737000BF006A14041030000B10780004004800AD
:10738000006F6682A817BF00780004009114840083
:107390000D0084001F0084004700AD0984000B002D
:1073A000780005004800656E646F6685B317BF00FE
:1073B00078000500911484004600AD090C00B8095E
:1073C000780004004800656E646361736587C717C1
:1073D000BF0078000400911484000B0087000410A3
:1073E0003000890A47000800B8094600F0FF041081
:1073F0003500480000233A02D817BF006A00630036
:10740000720082000E053000150030000E053500B8
:107410006200610716000E053500480000682382EF
:10742000ED17F21710000000006423820118F21714
:107430000A000000006F23820718F21708000000FE
:10744000006223820D18F2170200000000746882A7
:107450001318F21710000000007464821918F21754
:107460000A0000000024627566041F18C70060014E
:107470002F24627566052618C700640100616464E4
:107480002D63686172082C18BF0026182C1805009F
:107490003600780001002C18050075002C18F90D35
:1074A000480000243E24627566063418BF000F00B1
:1074B00026182C1805000C00A30E2C1805007500CA
:1074C0002C18F90D4800006E6578746368617208C5
:1074D0004618BF000A002200470006000E004900BF
:1074E0000D00310015000C0025000C003D0B1600AE
:1074F0005E0648006E657874686578075918BF00A5
:10750000591847001C0078001000960047000A0038
:107510005E065E06460006000B00570646000600A3
:1075200057065E064700DAFF48006765742D6865F8
:10753000782D62797465730D6F18BF00760029008D
:10754000000061006F1847003E0015006F18220010
:107550006F0F224F6464206E756D626572206F66D6
:10756000206865782064696769747320696E207388
:107570007472696E6700160078000400060D05003D
:1075800034184600C0FF4800006765742D636861C9
:1075900072088D18BF00A9060805300008074700CB
:1075A000100031007800010008053C00460008008A
:1075B0000B007800FFFF4800006765742D6573635A
:1075C000617065642D737472696E6712BA18BF00BA
:1075D0002D05300008053000050075002618F90D4E
:1075E0005D0075002C18F90D760022000000610086
:1075F0004618BA180A00A5008E0B47000A000B00B7
:1076000026182C18490076006E0000000D001F009F
:1076100047000E000B0078000A0034184600D8001E
:107620007600720000000D001F0047000E000B00E6
:1076300078000D0034184600BE007600740000008B
:107640000D001F0047000E000B00780009003418E1
:107650004600A4007600660000000D001F004700F1
:107660000E000B0078000C00341846008A007600EB
:107670006C0000000D001F0047000E000B0078009A
:107680000A003418460070007600620000000D0009
:107690001F0047000E000B00780008003418460059
:1076A00056007600210000000D001F0047000E006C
:1076B0000B0078000700341846003C0076005E009E
:1076C00000000D001F00470012000B00BA187800E0
:1076D0001F000200341846001E007600280000003B
:1076E0000D001F0047000A000B008D18460008001F
:1076F0000A0034180B004600F0FE48002281D7181B
:10770000BF00D7183305300047000400080F4800B9
:107710003E74797065057019BF000F00B30B0C0043
:107720003D00B30B0C00500048006C6D617267693E
:107730006E077C19C10068010000726D6172676993
:107740006E078A19C1006C0100003F6C696E650507
:107750009219BF00B00530000500921930002000DA
:1077600047000A004F008A193000C60B48003F63EB
:1077700072039919BF005D0099194800746F2D6359
:107780006F6C756D6E09AA19BF00B0053000060058
:10779000780001002C00C60B48000074616273740D
:1077A0006F707308B419C10070010000003F746F5E
:1077B0002D636F6C756D6E0AC319BF000F00050055
:1077C000921930002000470010000B004F008A196A
:1077D0003000C60B46000A00B00530000600C60B9C
:1077E0004800002E74616204CD19BF009219300068
:1077F000C319300005008A1930007F001A004400C8
:10780000B00530006F0B4700060044007D00C3192F
:1078100030008100EAFFCD194800776F726473056C
:10782000E519BF005D008A19350078004000921903
:10783000350078000E00C3193500090850063400E1
:10784000D313DF1347001E00CD0C0A0078001F0081
:107850000200E5195000BD0B4F0E4700040049001F
:107860004600E0FF4800776F72647305DF13BF00C6
:10787000011A4800002E32020000BF0058119D116D
:10788000CC11CC11A5115000BD0B4800002E3802C0
:107890002D1ABF009D117B157B157B157B157B1564
:1078A0007B157B157B158B155000BD0B4800642E96
:1078B0003203391ABF00570E7E000C00440031001D
:1078C0002D1A8000F8FF4800656D69742E054A1A6C
:1078D000BF0078007F0002000A00870E22004700E8
:1078E0000A000B0076002E0000004E004800646C79
:1078F0006E03581ABF0009080A00780008000C122D
:1079000078000200C60B780008008E064A1ABD0BEC
:107910000D000500780008004A1ABD0B7800100021
:10792000570E7E000C0044003100581A8000F8FF0A
:1079300048003F2E6E036A1ABF008E061F004700E4
:107940000E008300025C2F000B0046000800780048
:1079500002003C12BD0B48003F2E61038C1ABF0091
:107960008E061F0047000E008300017600000B000A
:1079700046000800780001003C124800006C2E68A8
:10798000656164069F1ABF000C000A007800F0FFD2
:1079900002000C0078000F00020078000A00C60BFD
:1079A000780010005D007F00140078000600C60B10
:1079B00044008C1A780004008100F0FFBD0B7800B1
:1079C00010005D007F000A0044009F1A8000FAFF4B
:1079D0001000050048006C2D646C6E05B31ABF00E2
:1079E00009080A00780008000C1278000200C60B93
:1079F0000A0078001000570E7F001000440030008D
:107A0000391A780004008100F4FFBD0B78001000E3
:107A1000570E7E000C0044003100581A8000F8FF19
:107A200048002E6865616405DF1ABF000C000A007B
:107A30007800F0FF02000C0078000F0002007800D0
:107A40000A00C60B780008005D007F000A004400B1
:107A50008C1A8000FAFFBD0B780010007800080037
:107A60007F000A0044008C1A8000FAFFBD0B7800EA
:107A700010005D007F000A0044009F1A8000FAFF9A
:107A80001000050048000064756D7004011ABF0005
:107A90000E05300011001709051B0A0022004700DF
:107AA00004002500570E7F00120044006A1A4F0E92
:107AB0007C00780010008100F2FF0E0535004800C0
:107AC0006C64756D7005371BBF000915B31A570E2E
:107AD0007E0012004400DF1A4F0E7C007800100078
:107AE0008100F2FF2715480000647502541BBF0097
:107AF0000A0078004000371B78004000050048006D
:107B00006373656172636807671BBF000C008E06B4
:107B1000760B47000A00A0060B00570649000A0032
:107B20003100780003001200890A47000800DB0AD0
:107B30004600DCFF0E000E005E06480077736561AC
:107B400072636807751BBF001000401111000C0024
:107B50008E06760B47000A00A0060B005706490068
:107B60000A003200780003001200890A470008006A
:107B7000E20A4600DCFF0E000E005E064800747349
:107B8000656172636807931BBF000C008E06760B5D
:107B900047000A00A0060B00570649000A003400FF
:107BA000780003001200890A47000A002500070C2C
:107BB0004600DAFF0E000E005E0648006E73656137
:107BC00072636807B41BBF000C008E06760B47007B
:107BD0000A00A0060B00570649000A003000780092
:107BE00003001200890A47000A002500070C46001E
:107BF000DAFF0E000E005E064800776F72642D6299
:107C00006F756E64730BD31BBF00510075000202C9
:107C10000D005E00B41B2200470004005E00480017
:107C20006669747331363F07F41BBF0078000F009C
:107C300009007800FFFF5D006C0C4800006E706169
:107C40007463682D7431360A051CBF00F41B0C00E8
:107C50008E06760B6F0F0D43616E27742066696E7A
:107C60006420697400000A003000780003001200EC
:107C70001F0047000A000E000E00350049000A00F0
:107C80003400750016031F0047005200960C0A00CE
:107C90007C117800030012001F00470040000E0016
:107CA0000E000D00051C47000600370049000B00C0
:107CB0002C12830023646F6573206E6F74206669D5
:107CC0007420696E2074686520617661696C6162F8
:107CD0006C6520737061636500005A002500070C15
:107CE00046006EFF4800286E706174636807151CBB
:107CF000BF00151C48002877706174636807681C12
:107D0000BF00F41B931B4700080037004600180013
:107D1000830010436F756C646E27742066696E640F
:107D2000206974000B0048000028706174636806C5
:107D3000701CBF00F41BB41B47000800390046004C
:107D40001800830010436F756C646E277420666999
:107D50006E64206974000B004800006E70617463EB
:107D60006806891CBF007C09681C480000777061A8
:107D700074636806A21CBF007C09701C4800706117
:107D800074636805AB1CBF007C097C097C09891CF5
:107D90004800667075736805B31CBF004800006535
:107DA0002E02BD1CBF0048000028666C6974657215
:107DB000616C290AC21CBF0048002E6573635B0515
:107DC000CB1CBF0078001B00F41576005B000000A0
:107DD000F4154800002E6573635B7806D11CBF0064
:107DE000D11CF41548007075742D6E05DF1CBF00A2
:107DF000191518120016271548002E6573635B6E5F
:107E00007807E71CBF00D11C0D00E71CF4154800E3
:107E1000006C65667404F21CBF007600440000002C
:107E2000DF1C7800FFFFB0053C00480072696768FE
:107E30007405FC1CBF00760043000000DF1C7800C6
:107E40000100B0053C004800007570020A1DBF002B
:107E5000760041000000DF1C7800FFFFB6053C0003
:107E6000480000646F776E04171DBF007600420063
:107E70000000DF1C78000100B6053C004800696E78
:107E8000736572742D636861720B251DBF007600E7
:107E900040000000DF1CF415480064656C657465E3
:107EA0002D636861720B361DBF0076005000000024
:107EB000DF1C48006B696C6C2D6C696E6509441D94
:107EC000BF0076004B000000DF1C48006B696C6C43
:107ED0002D73637265656E0B501DBF0076004A00FE
:107EE0000000DF1C4800696E736572742D6C696E4A
:107EF000650B5D1DBF0076004C000000DF1C4800D4
:107F000064656C6574652D6C696E650B6A1DBF00D8
:107F100076004D000000DF1C4800696E76657273C4
:107F2000652D766964656F0D771DBF00760037009B
:107F30000000DF1C76006D000000F41548006C6541
:107F400066747305851DBF00760044000000F21CB6
:107F50002F00B0053C004800007269676874730622
:107F6000931DBF00760043000000F21CB0053C00EA
:107F7000480075707303A11DBF007600410000002A
:107F8000F21C2F00B6053C004800646F776E730545
:107F9000AC1DBF00760042000000F21CB6053C009C
:107FA00048000063616E63656C06B91DBF00760012
:107FB0006D000000DF1C4800006E6F742D6461725C
:107FC0006B08C61DBF00760032000000DF1C760083
:107FD00037000000F41576006D000000F41548002D
:107FE0006C6967687405D21DC400740100000064E8
:107FF00061726B04E41DC4007801000061742D7887
:108000007905EB1DBF008E06B6053500B0053500BD
:10801000D11C2500E71C76003B000000F41525006C
:10802000E71C760048000000F41548000070616706
:108030006504F21DBF005D005D00F21D5D1D48007E
:1080400000616E73692D636F6C6F72733F0C0A1E53
:10805000C7007C0100636F6C6F723A06181EBF0088
:108060006A00DD0E8200181E47001400D11C41007A
:10807000001676006D000000F415460004000B00A9
:1080800048000064656661756C742D636F6C6F7277
:10809000730E1F1E231E01300000006272696768A4
:1080A00074063A1E231E0131000064696D03421EEE
:1080B000231E01320000756E6465726C696E65097D
:1080C000481E231E01340000626C61636B2D6C65D9
:1080D00074746572730D511E231E02333000726575
:1080E000642D6C6574746572730B5C1E231E023301
:1080F0003100677265656E2D6C6574746572730D01
:10810000661E231E023332000079656C6C6F772D7A
:108110006C6574746572730E711E231E0233330016
:1081200000626C75652D6C6574746572730C7D1ED0
:10813000231E023334006D6167656E74612D6C65BA
:1081400074746572730F881E231E0233350000633A
:1081500079616E2D6C6574746572730C941E231EA8
:108160000233360077686974652D6C6574746572C6
:10817000730D9F1E231E0233370000626C61636B18
:108180002D73637265656E0CAA1E231E02343000C7
:10819000007265642D73637265656E0AB51E231ED9
:1081A0000234310000677265656E2D736372656518
:1081B0006E0CBF1E231E0234320079656C6C6F7723
:1081C0002D73637265656E0DCA1E231E0234330063
:1081D000626C75652D73637265656E0BD51E231E0B
:1081E00002343400006D6167656E74612D736372D3
:1081F00065656E0EDF1E231E023435006379616EE5
:108200002D73637265656E0BEB1E231E0234360000
:108210000077686974652D73637265656E0CF51E71
:10822000231E0234370032636F6E7374616E7409FB
:10823000001FBF006A006300630082000A00430061
:1082400030000C003000480000326C6974657261C7
:108250006C88091FBF000C00740674064800327653
:1082600061726961626C65091A1FBF006A005D0076
:1082700063005D006300480064303C03251FBF00BD
:108280000E002100480000643C022F1FBF001000B8
:108290000C008E06890A470004009606A0061E0000
:1082A0004800006461627304361FBF008E062F1FF2
:1082B0004700040091004800643E7303451FBF005F
:1082C0000B0048000028642E29044F1FBF000F0038
:1082D000451F9D11F0111000B111A5114800006457
:1082E0002E02561FBF00561F5000BD0B48002875B8
:1082F000642E2905621FBF009D11F0111000A51109
:10830000480075642E036B1FBF006B1F5000BD0B30
:1083100048000075642E7204741FBF0015006B1FA7
:1083200016000D000600C60B5000480000643D0218
:108330007D1FBF009200E911480064322A03891FA3
:10834000BF00450B0D0021004700040025000C0074
:10835000450B0C00480064322F03901FBF000A0039
:108360002B000C00780001000200100078000100D2
:10837000FF0C0C0078001F00060D03000C004800E5
:1083800000646D6178049E1FBF004E0B4E0B361FBC
:10839000470004009606A006480000646D696E045C
:1083A000B41FBF004E0B4E0B361F220047000400C7
:1083B0009606A0064800006D2B02C11FBF00511198
:1083C000930048000032726F7404CE1FBF00180083
:1083D000960619009606480064753C03D61FBF0038
:1083E00010000C008E06890A470004009606A006BD
:1083F000240048006C6273706C697407DF1FBF0053
:108400000A007800FF0002000C00780008000C0D44
:108410000A007800FF0002000C00780008000C0D34
:108420000A007800FF0002000C00780008000C0D24
:108430007800FF0002004800776273706C6974076F
:10844000EF1FBF000A007800FF0002000C00780058
:1084500008000C0D7800FF00020048006C77737074
:108460006C6974071120BF000A007700FFFF00004D
:1084700002000C00780010000C0D7700FFFF0000D8
:108480000200480000626C6A6F696E062320BF001C
:1084900078000800060D050078000800060D0500AC
:1084A00078000800060D050048000062776A6F69D1
:1084B0006E063720BF0078000800060D0500480052
:1084C00000776C6A6F696E064A20BF007800100062
:1084D000F70C030048000066696E642D636661084E
:1084E0005520BF00370B06000A00130DB4041F000F
:1084F0004700F2FF48006973646566657207612092
:10850000C4008001000000697375736572067020F5
:10851000C30084010000006973636F6E7374616E41
:10852000740A7820C0000000000000697376617250
:108530006961626C650A8220C100880100003E7496
:108540006172676574078C20BF00960C0A003B00BF
:108550000500480000636F6465049420BF00480074
:108560007072696D6974697665099E20BF00480064
:10857000646566696E657207A620BF000A00130D68
:108580000A00A1001E0047000A00A0067500A620F0
:1085900049000A00F4048E0B4700BE000E00B4042C
:1085A0000D001F0047000C000B007500A4024600E0
:1085B000A400BE040D001F0047000C000B00750056
:1085C000AB0246009000C8040D001F0047000C00DD
:1085D0000B007500B70246007C00D1040D001F009F
:1085E00047000C000B007500BD0246006800D9046E
:1085F0000D001F0047000C000B007500B002460084
:108600005400E1040D001F0047000C000B00750032
:10861000820D46004000EC040D001F0047000C00D6
:108620000B007500DF1246002C00F4040D001F0043
:1086300047000C000B0075009E2046001800FC044B
:108640000D001F0047000C000B007500E00D4600F8
:1086500004000B00460008000B00340061204800B5
:108660003E636F646505AD20BF00510048003E6465
:10867000617461052421BF000A0051000C00130D34
:10868000C8040D001F0047000A000B00300D460013
:108690004C00D9040D001F0047000A000B00300DEC
:1086A00046003A00E1040D001F0047000A000B00DD
:1086B000300D46002800EC040D001F0047000A00A2
:1086C0000B00300D46001600FC040D001F00470093
:1086D0000A000B00300D460004000B004800002883
:1086E0006F6629042B21BF00480028656E646F6601
:1086F00029076321BF00480028656E6463617365C4
:1087000029096A21BF00480000696E2D64696374FD
:10871000696F6E6172793F0E7221BF009D005E002D
:108720005F0C48006C6F6F702D656E643F097D2192
:10873000BF000B005706480000696E6469726563EC
:10874000742D63616C6C3F0E8821BF000B005706CF
:1087500048000072736C6973748695214210A006FC
:10876000FFFFFFFF756E627567059E21BF005D000C
:1087700031063500480000756E616C69676E65648E
:108780002D77400CA621BF000A0031000C00250007
:1087900031004A20480000756E616C69676E65643F
:1087A0002D6C400CB321BF001500170031001700DD
:1087B0002500310017002600310016007800030064
:1087C0000500310037204800756E616C69676E6581
:1087D000642D400BC321BF00C32148000064400248
:1087E000DB21BF00590B48000074616C69676E653E
:1087F0006488E1214210070CFFFFFFFF002B737418
:108800007204EA21BF00410005002500070C480062
:10881000006E2E02F221BF002C124800656D6974B3
:108820002E05FB21BF0078007F0002000A00870EA2
:108830002200470008000B0078002E004E00480080
:10884000656D69742E6C6E070222BF00570E7E00A4
:108850000C004400310002228000F8FF4800287319
:10886000656529051522C4008C010000002F706F7A
:10887000736974696F6E730A051BC000600900009C
:10888000706F736974696F6E73092D22B61690014B
:108890000000600900000000656E642D706F736950
:1088A00074696F6E730D3622C700940100696E699A
:1088B000742D706F736974696F6E730E4422BF00FC
:1088C000362275004422F90D480066696E642D70E9
:1088D0006F736974696F6E0D4F22BF004422362298
:1088E0007E0024004400590B0E000D001F004700BD
:1088F0000C000B0044005706E21449007800020007
:10890000A5148100E0FF0B005E0648006465636FFC
:108910006D70696C65722D69700D5D22C7009801DC
:10892000006164642D706F736974696F6E0C7E22D0
:10893000BF007E225D2247004200442236222D22C3
:1089400005006F0B6F0F224465636F6D70696C6576
:108950007220706F736974696F6E207461626C65E8
:10896000206F766572666C6F770044220A0078008B
:1089700002002E0B75004422F90DB0053000B6053B
:10898000300055207E221000640B480069703E7054
:108990006F736974696F6E0B8822BF005D22470098
:1089A00008005E0646000A00590B0B0023205706FC
:1089B000480069702D7365742D637572736F720D45
:1089C000BD22BF00BD22220047000400F21D480066
:1089D00000696E64656E7406D122C4009C010000BB
:1089E0000028696E64656E742908DD22BF008A194B
:1089F0003000B005300006005D002C00C60B4800BA
:108A00002B696E64656E7407E622BF007800030070
:108A10008A193C004F0048002D696E64656E74072A
:108A2000F522BF0009087800FDFF8A193C004800C4
:108A3000006372222E040123BF000A009919DD226F
:108A40008822941E5000C61D48002E2E22830C231F
:108A5000BF00701984000C2348006F75740318233D
:108A6000BF004F0083001A7375627363726970747C
:108A7000206F7574206F662072616E6765206F6E5F
:108A800020000A00EE0CDC0C83000A2020206D611F
:108A90007820697320008B128300092020207472D3
:108AA0006965642000002C12950848006D61700310
:108AB0002023BF008E063000240047000C00280B46
:108AC0000C002E0B4600040020234800006D61704E
:108AD000746F6B656E084923BF008E06300024005A
:108AE00047001000280B0C009F00070005004600FF
:108AF000040020234800636173653A052322BF0008
:108B00006A00630099006A0682005C2334004A0010
:108B10004800746173736F636961746976653A0DB7
:108B20006F23BF006A00630082000A0030000A0061
:108B300015001100280B16005D007F001E008E0638
:108B400034001F0047000E00A0060B0044005D002B
:108B50005D007D00960C8000E6FFA0064800002323
:108B6000656E7472696573085C23BF005100300044
:108B700048006E756C6C64697307A523BF000B0019
:108B80008300113C6E6F20646973617373656D625D
:108B90006C65723E00004800646973617373656DB3
:108BA000626C650BAE23C400A00100002F627265E9
:108BB000616B7307C323C00040010000006272654F
:108BC000616B7306CB23B616A401000040010000C0
:108BD000362200656E642D627265616B730AD32361
:108BE000C100A801000000627265616B2D7479708C
:108BF000650AE023C100AC01000000627265616B90
:108C00002D616464720AEA23C100B0010000776834
:108C10006572652D627265616B0BF423C100B4014E
:108C20000000006E6578742D627265616B0AFE2328
:108C3000BF007800FFFFF4233500E0233000D3238A
:108C40007E002E004400590B0D00F4233000240058
:108C500047001400EA233500F42335004400FE23C6
:108C6000350046000400A0061F0B450B8100D6FF0F
:108C7000F42330007800FFFF890A470010007800D5
:108C8000FFFF7800FFFFFE233000640B4800666F93
:108C900072776172642D6272616E63683F0F08249F
:108CA000BF000A0094202400480000626172652D14
:108CB00069663F084024BF00A00006009F00060030
:108CC0000A0034000A007500F6011F0047000A0080
:108CD0000B000B00570649007500FC011F00470000
:108CE00008004024460006000B005E06480000779E
:108CF00068696C653F064B24BF009420A000060005
:108D00009F0006000A0034007500F6011F004700AE
:108D10000A0040242200460006000B0057064800C7
:108D2000002E626567696E066C24BF00FF0E066246
:108D30006567696E20000C23F52248002E74686573
:108D40006E058524BF000123FF0E047468656E0064
:108D50000C234F0048000070662D656E6406922457
:108D6000C700B80100657874656E7406A024C10060
:108D7000BC0100002B657874656E7407A724BF00E2
:108D8000A7243000520CA724350048002B627261E2
:108D90006E636807AF24BF00960CA0000500480072
:108DA000002E656E646F6606BB24BF00FF0E05656E
:108DB0006E646F6600000C234F00BB244800002E39
:108DC000656E646361736508C524BF00FF0E0765A7
:108DD0006E646361736500000C234F00960C4800BD
:108DE0006164642D627265616B09D524BF00E02364
:108DF0003000D323CB2305006F0B6F0F194465633D
:108E00006F6D70696C6572207461626C65206F763D
:108E10006572666C6F770000E0233000D32320007A
:108E2000470036000D00E02330001F0B450B060005
:108E300015001700590B7500C5241F0011001F00F5
:108E40000200470010001700590B96061600640B2D
:108E50004600060016000B00E0233000640B1F0BD9
:108E6000450BE0233C004800003F6164642D6272C2
:108E700065616B0AE624BF000D00E0233000D323B8
:108E80007E001E000A004400590B0B001F00470023
:108E900008000B005D007D001F0B450B8100E6FF05
:108EA00047000800E62446000400A006480073635B
:108EB000616E2D6F66072B25BF000A0094200A0003
:108EC000AF24A00006009F0006000A007500C5241C
:108ED000E6247500D5242B25BB2448007363616EFE
:108EE0002D6272616E63680B4C25BF000A000A0098
:108EF00040244700200094200A00AF240A004B249D
:108F000047000C0075009224E624460004000B0084
:108F100046000A00942075008524E624BB244800FE
:108F2000736B69702D63686172096525BF00960CCB
:108F3000960C48007363616E2D756E6E6573740BCD
:108F40008625BF000A00A7243000870B47001000C9
:108F5000960C7500A024F90D5D0046000400960CE7
:108F60004800007363616E2D646F65733E0A91253E
:108F7000BF00960C48002E6272616E636807A825D8
:108F8000BF000A004024470014000123FF0E0465BF
:108F90006C7365000C23F522460012000123FF0EBE
:108FA00006726570656174000C234F00BB24480095
:108FB000002E3F6272616E636808B025BF000A0030
:108FC000402447002C000A006C24470016000123AF
:108FD000FF0E057768696C6500000C23F5224600DA
:108FE0000C00FF0E026966000C23F52246001200F9
:108FF0000123FF0E06756E74696C20000C234F0070
:10900000BB2448002E646F03CE25BF00FF0E06640C
:109010006F20202020000C23F522BB244800002EC6
:109020003F646F04F525BF00FF0E063F646F2020EC
:1090300020000C23F522BB2448002E6C6F6F7005B6
:109040000326BF000123FF0E066C6F6F7020200007
:109050000C234F00BB244800002E2B6C6F6F700652
:109060001126BF000123FF0E062B6C6F6F702000CE
:109070000C234F00BB2448002E6F66032126BF003F
:10908000FF0E056F6620202000000C23BB24480043
:1090900000636865636B2D706F7374706F6E650E1F
:1090A0002F26BF000A00C10C47001000FF0E0870F9
:1090B0006F7374706F6E65000C23480000707574D8
:1090C00022044126BF007600220000004E00BD0BA6
:1090D00048000063776F72642D6E616D650A5226D9
:1090E000BF000A003400CD0C0C0025000C007800F5
:1090F000020006001000960C110078000200120019
:109100004100960648007479706523056026BF000B
:10911000570E7E002800440031000A00780020002D
:109120001E00470012000B00711E83000123000087
:10913000661E460004004E008000DCFF4800002E42
:10914000737472696E672D7461696C0C7726BF0049
:109150007800020012000D000500780003000500F1
:1091600099190C23BD0B661E7726941E76002200EB
:1091700000004E00BD0BC61D48000070726574747F
:10918000792D2E089726BF000E05300078000A00C2
:109190001F0047000800181246000400FB110A00D7
:1091A0007800030005009919DD228822711E0E0542
:1091B000300078000A000D001F0047000E000B0071
:1091C00083000123000046004E00780010000D00CF
:1091D0001F0047000E000B00830001240000460022
:1091E0003600780008000D001F00470010000B003B
:1091F0008300036F2320000046001C00780002005B
:109200000D001F0047000E000B0083000125000029
:10921000460004000B005000C61DBD0B48002E6325
:109220006F6D70696C656409B326BF000A00340075
:109230004126CD0C5000BD0B960C48002E776F7266
:1092400064050527BF00DD220A0034004126CD0C4D
:109250000A00991988225000BD0B960C4800736BC8
:1092600069702D776F7264091227BF00960C480051
:109270002E696E6C696E65072527BF00960C0A0083
:10928000DB21B326280B4800736B69702D696E6C67
:10929000696E650B2D27BF00960C280B48002E77B2
:1092A0006C6974053B27BF00960C0A00B321B326F6
:1092B000E20A4800736B69702D776C697409432763
:1092C000BF00960CE20A48002E666C6974055027B0
:1092D000BF00960C15001600E90AE90A48002E6C3A
:1092E0006C6974055827BF00960C0A00C321B32689
:1092F000E90A4800736B69702D6C6C697409632707
:10930000BF00960CE90A4800736B69702D627261A8
:109310006E63680B7027BF00BB244800002E636F8C
:109320006D70696C65087B27BF00FF0E08636F6D69
:1093300070696C6520000C23960C052748000073AB
:109340006B69702D636F6D70696C650C8427BF004D
:10935000960C960C4800736B69702D737472696E6D
:10936000670B9727BF00960CF2214800002E5B2761
:109370005D04A227BF00960CFF0E045B275D200052
:109380000C230A003400DC0C960C480000736B6957
:10939000702D5B275D08AA27BF00960C960C48002D
:1093A0002E746F03BC27BF00FF0E03746F200000F4
:1093B0000C23960C0A003400DC0C960C48002E732B
:1093C0007472696E6707C327BF0060269726F22173
:1093D0004800002E646F65733E06D427BF00FF0E61
:1093E00006646F65733E20000C23960C48002E75B2
:1093F0006E6E65737407DE27BF000A00A724300075
:10940000870B47001A0009085D008A193500FF0E16
:10941000013B00000C230B005D0046001000FF0E16
:1094200005657869742000000C23960C480064756B
:109430006D6D7905EC27BF0048002E6368617205E9
:109440000B28BF00FF0E012700000C23960C0A001A
:1094500030004E00BD0B280B4800236465636F6D20
:10946000702D636C61737365730F1128C000170052
:109470000000657865637574696F6E2D636C617348
:10948000730F262885231700000077004700460049
:10949000800081007F00840083006F0F0B2848004C
:1094A000FF0E7E0082007600CB1C750063216A21CE
:1094B0007221F70E78000B28002E657865637574AD
:1094C000696F6E2D636C61737310322875231800F9
:1094D00000002D27CE25B02511262126F52584272D
:1094E000D427D4270B28EC27D4270326DE271128DE
:1094F0005827AA272F26C524D524D42743270B284D
:1095000012274800646F2D7363616E075628752318
:10951000180000003B27652565257B277B277B27D7
:109520009727A227A2270B289125A2277B27A825CA
:1095300086257027BC274C257B272527A2277B273C
:109540000B28252748007363616E2D706607772806
:10955000BF000A00A7243500D323E02335000A000A
:109560003400322877280A0022004700F2FF0B005F
:109570004800002E746F6B656E068123BF000A00E1
:1095800034003228562848002E706603AE28BF00EB
:109590004F220A0098280824780003008A19350011
:1095A000DD220A0075007E22F90DAA19F42330008D
:1095B0000D001F0047001A00EA2330004A0008246B
:1095C000F42330000D00890A4700EEFF4600040036
:1095D000AE280A0022004F0E4700060096155B00D9
:1095E0004700C0FF0B004800002E696D6D6564697F
:1095F0006174650A9828BF00C10C47001200FF0E75
:1096000009696D6D65646961746500000C2348002B
:10961000002E646566696E657208EB28BF00941EB3
:10962000DC0C0A00881EDC0CC61D480064756D70D9
:109630002D626F647909FE28BF0009150A00300009
:10964000B32678000200C60B780008001522271503
:109650004800002E3A020C29BF00FE284F0051009E
:10966000B728480064656275672D736565091C2914
:10967000BF0061207500A4021C2948002E636F6E94
:109680007374616E74092829BF000D002B2130000E
:10969000B326FE280B004800002E32636F6E7374F1
:1096A000616E740A3429BF000D002B210A003000BE
:1096B000B326280B3000B326FE280B0048002E7678
:1096C0006F636162756C6172790B4329BF00FE287C
:1096D0000B0048002E636F6465055629BF00FE2805
:1096E0002421C32348002E7661726961626C65098A
:1096F0005E29BF000D002B21FB21FE288300087688
:10970000616C7565203D20002B213000B326480098
:109710002E637265617465076929BF000D005100F1
:10972000FB21FE2883000876616C7565203D2000D2
:1097300051000C2948002E75736572057D29BF0004
:109740000D0051003000FB21FE28830009207661C6
:109750006C7565203D2000002B213000B3264800A9
:10976000002E6465666572068F29BF00FE2883009F
:109770000369732000004F002B213400232248008E
:10978000002E616C69617306A529BF00FE28510097
:109790003400DC0C4800002E76616C756506B52936
:1097A000BF000C002B213000B326FE284800002EFD
:1097B0006F7468657206C029BF00FE2851008300DF
:1097C0000A20202028426F64793A20000C29830067
:1097D0000320292000004F00480063662C03CC2999
:1097E000BF007C099D0D480023646566696E69743D
:1097F000696F6E2D636C617373657313E029C0002C
:109800000C00000000646566696E6974696F6E2DF6
:10981000636C61737310EF2985230C0000006600F0
:10982000670069006800820D6A00DF124D10E00DCC
:10983000091F9E200B282E646566696E6974696F26
:109840006E2D636C61737311FC2975230D0000008C
:109850001C29342969298F29A5297D295629B5294B
:10986000C02943295E290B28CC29480000696E7362
:1098700074616C6C2D6465636F6D702D64656669D1
:109880006E657216B728BF0075000B287500152A83
:10989000891C75000B287500FC295100280B0A0053
:1098A00078000C009D0CB41B0B00390048002828E0
:1098B00073656505152ABF007800300092193500E0
:1098C0000A000A00AD200A00FC29152AEB28090825
:1098D000480073656503332ABF007C0975002322A5
:1098E0001408470004000B00480074726163652D82
:1098F000746F6F6C732E660D5C2AC2000072656116
:10990000736F6E61626C652D69703F0E4B2ABF00EC
:109910000A009D005E006C0C47000C000A00070C5A
:109920001F00460006000B005706480070726F6269
:1099300061626C792D6366613F0D772ABF00772ADB
:1099400048002E63757272656E742D776F72640DA8
:109950008E2ABF006120DC0C4800002E6C617374FD
:109960002D65786563757465640E992ABF009F0044
:10997000060034000A008E2A47000800DC0C46006E
:109980000A000B008300023F3F0048002E63616C19
:109990006C657207A62ABF0078001200B419830014
:1099A0000C43616C6C65642066726F6D20000A0068
:1099B000992A78003800B4198300036174200000EC
:1099C0002C124800002E63616C6C73066D2ABF0078
:1099D000750050068E065E00B41B470010000A009A
:1099E000BB2A4F000E00960C4600EAFFA006480076
:1099F00000726571756972657308D72ABF007609B0
:109A0000470008000B0046000400F70848006E6598
:109A100065647385EE2ABF00760947000C000B00D1
:109A20006200A00646000800A0066200F708480091
:109A3000005C6E6565647386FB2ABF00760947008B
:109A40000A000B00340946000400A00648007369B0
:109A500066742D737472696E670BBB2AC100C001F6
:109A600000007673696674051E2BBF000908830029
:109A700011202020496E20766F636162756C6172DF
:109A8000792000000A00DC0C4F00D3131800DF130C
:109A900047003A000A00CD0C8E061A00A6004700C7
:109AA0002400A006AA198300012800001000FB1161
:109AB0005000830002292000500078000300C60BEC
:109AC00046000600A006FF144600C4FF1900A006C9
:109AD00048002473696674050D2BBF00E505071364
:109AE0004700120015008E061700252B16001B13C9
:109AF0004600ECFFA006480073696674696E67074C
:109B00005D2BBF006A095D2B480024617272617988
:109B10003A07712BBF006A005D0063009D009D0D38
:109B200082008E0630005D000C005F0C22006F0F7B
:109B30001F537472696E6720617272617920696E59
:109B4000646578206F7574206F662072616E67653A
:109B50000000280B34000C009D0C3400410048002C
:109B60003B246172726179077A2BBF005E00130C8F
:109B7000E60C5100280B5E000D003900960C8E0695
:109B8000200047000E000A009D0DD20EA0064600E0
:109B9000EEFFA006E60C51000A00280B34005E0020
:109BA0000C0006009F008D000C003500480000638B
:109BB00063616C6C7306A52BFB12C401F4137B016B
:109BC0000000BF005D006A090B0031000A0076004A
:109BD0002D0000001F004700EEFF0B000A004700A9
:109BE00008002B094600F6FF0B0076002D00000050
:109BF0002B096A090B0031000A0076007D00000085
:109C0000890A470008002B094600E8FF5D002B0980
:109C10000B00130C69134800006363616C6C3A0617
:109C2000CC2BBF006A0063005D005E00360031137C
:109C3000CC2B82000A00280B0C003000A300480047
:109C40000069703E746F6B656E08012CBF009F0049
:109C500006004800002E74726163656C696E650AC7
:109C6000252BBF0009150A00772A47000E000A00BD
:109C7000A62A162CBB2A46000800780009000C1200
:109C80004F002715480000287273747261636508DD
:109C9000212CBF007E00120044003000212C4F0E0A
:109CA0007C001F0B8100F2FF4800727374726163C5
:109CB0006507162CBF00890097053000800B470010
:109CC000260083001652657475726E2053746163AA
:109CD0006B20556E646572666C6F77009705300077
:109CE0008A0046000A00970530008900392C480098
:109CF00000617472616365064A2CBF008300144CD6
:109D00006173742061626F7274206F722074687264
:109D10006F773A004F00AA053000A3053000392CB8
:109D20004800656E7669726F6E6D656E740B6D2C92
:109D3000FB12C801CC2B002F616C69676E06000016
:109D4000C000020000002F6368617205902CC00003
:109D5000010000002F636F756E7465642D7374725B
:109D6000696E670F972CC000FF0000002F646174BC
:109D7000612D73706163650BA32CC00000000200AD
:109D80002F686F6C6405AD2CC00064000000002FCC
:109D900070616404B42CBF009D00AD2C0500B30BB2
:109DA00006004800002F74696204BB2CC0008400C8
:109DB0000000616464726573732D756E69742D6241
:109DC00069747311C62CC0000800000000636F7234
:109DD0006504D32CC000FFFFFFFF00636F72652D89
:109DE00065787408DA2CC000FFFFFFFF00646F7510
:109DF000626C6506E32CC000FFFFFFFF00646F7517
:109E0000626C652D6578740AEB2CC000FFFFFFFFC4
:109E10000066696C6504F52CC000FFFFFFFF00665B
:109E2000696C652D65787408FC2CC000FFFFFFFF8E
:109E300000666C6F6174696E6708052DC000FFFFD6
:109E4000FFFF00666C6F6174696E672D6578740C36
:109E50000E2DC000FFFFFFFF00666C6F6174696E1E
:109E6000672D737461636B0E192DC0001400000020
:109E70000066756C6C04252DC000FFFFFFFF006CB1
:109E80006F63616C73062C2DC000FFFFFFFF006C39
:109E90006F63616C732D6578740A342DC000FFFF09
:109EA000FFFF6D61782D6E053E2DC000FFFFFF7F27
:109EB0006D61782D7505452DC000FFFFFFFF6D61B9
:109EC000782D64054C2DC000FFFFFF7F006D617889
:109ED0002D756406532DC000FFFFFFFF006D656DFB
:109EE0006F72792D616C6C6F630C5B2DC000FFFF8E
:109EF000FFFF006D656D6F72792D616C6C6F632D66
:109F000065787410662DC000000000000072657452
:109F100075726E2D737461636B2D63656C6C731257
:109F2000732DC00064000000007365617263682DCA
:109F30006F726465720C812DC000FFFFFFFF00731C
:109F400065617263682D6F726465722D6578741037
:109F50008C2DC000FFFFFFFF737461636B2D636581
:109F60006C6C730B992DC000640000000073747258
:109F7000696E6706A32DC000FFFFFFFF00737472B8
:109F8000696E672D6578740AAB2DC000FFFFFFFF77
:109F900000656E7669726F6E6D656E743F0C882C0D
:109FA000BF007500882C550047000A004A005E0675
:109FB0004600040057064800006D61726B6572062A
:109FC000C02DBF006A0003053000630082000A0054
:109FD000300003053500EE0C23144800746F3F0376
:109FE000D12DC100CC01000000646F2D6C6F636146
:109FF0006C08E12DBF007406E12D300047000A0017
:10A000008400AD00460006008400AC00E12D410C48
:10A010004800286C6F63616C2907EA2DBF000A00B5
:10A0200047001000160630007500EA2DB00046000B
:10A030000E00A0061606300074068400AE0048002C
:10A0400000746F82FE2DBF000805300015007C09EA
:10A0500016000805350075005F0434001F00470036
:10A060000A00E12D490C46000400280E48006C6FE0
:10A0700063616C85132EBF006200FE2D48000065F1
:10A080006E642D6C6F63616C738A2B2EBF005D0054
:10A090005D00FE2D48006578616D706C6507362E99
:10A0A000BF0078000100AE0078000000AC000A009C
:10A0B00078000000AC0007000A0078000000AC0047
:10A0C000070048006C6F63616C737C87402EBF0093
:10A0D00062000D00310076007C00000006000D00DB
:10A0E000780001000600030047000800FE2D46002E
:10A0F000E0FFA0065D005D00FE2D48000078310203
:10A10000572EBF0078000100AE0078000000AC00C0
:10A110000A0078000000AC0007000A007800000088
:10A12000AC0007004800006C6F63616C2306712E61
:10A13000C100D0010000006C6F636E616D65730833
:10A14000882EB616D401000000010000D323003E83
:10A150006C6F636E616D6508912EBF007800200002
:10A160000700912E05004800003B7365656E3F06B1
:10A170009D2EC100D8010000002D7365656E3F065D
:10A18000A92EC100DC01000000736176652D6C6FA3
:10A1900063616C0AB12EBF00B12E30004700080089
:10A1A000A00646001E00A92E3000470006008400CD
:10A1B0005706882E30009D2EB40E78000100882EA0
:10A1C0003C004800006465636C6172652D6C6F63D0
:10A1D000616C730EBB2EBF00882E30001400470048
:10A1E0001C001400470010003D0B0A009D2E41008A
:10A1F000FE2D4600EEFF5D005D00FE2D48007B81D8
:10A20000DB2EBF00B12E410CA92E410C882E410C33
:10A2100062000D00310076007D0000000D001F007F
:10A2200047000C000B00A0065E06460044007600C6
:10A230003B0000000D001F00470010000B00A92E7E
:10A24000490CA00657064600280076002D000000A5
:10A250000D001F00470010000B00B12E490CA00696
:10A26000570646000C0057060C009606BB2E0B0046
:10A2700047009EFFDB2E480000783202F12EBF001F
:10A2800078000100AE0078000000AC000A00780001
:10A290000000AC0007000A0078000000AC000700D6
:10A2A0004800007363726F6C6C696E672D64656241
:10A2B00075673F102F2FC700E001737465703F056D
:10A2C000392CC100E401000072657303512FC100F5
:10A2D000E801000000646973706C617965642D7831
:10A2E000740C572FC700EC01666F7263652D7265A1
:10A2F000646973706C61790F622FBF007800FFFF93
:10A300007500622FF90D480028646562756729079A
:10A310006D2FBF00A621780001003B0635003606F0
:10A32000350031063500512F490C6D2F4800277537
:10A330006E6E65737407792FBF009828A0244800BB
:10A340007365742D3C6970078C2FBF003106350092
:10A350003106300036063000870B47000C0031060E
:10A3600030008C2F36063500480000646566657243
:10A370003F064B2FBF00440D75001802440D1F000F
:10A380004800007265736F6C76652D646566657252
:10A39000730EAA2FC400F001000000287265736FCD
:10A3A0006C76652D6465666572732910BA2FBF00DF
:10A3B0000A00AA2F470008004B004600F4FF48009F
:10A3C0000028646562756706C72FBF00BA2F0A00B0
:10A3D000AD207500A402890A6F0F164E6F742061BC
:10A3E00020636F6C6F6E20646566696E6974696F57
:10A3F0006E0051000A008C2F792F480000646562BE
:10A4000075672D6D6508D52FBF001C006120D52F05
:10A4100048000064656275672806F42FBF001C00C1
:10A420000A008C2F792F4800002964656275670641
:10A43000FE2FBF001C0036063500480064656275BB
:10A44000672D6F6666090930BF00A6214800757048
:10A450003103952FBF00280B0A0097053000890AA9
:10A4600047005C000A0030000A007D2147004A00D6
:10A470000A008821470008000B00460038006120D0
:10A480000A009521470008000B00460028000E0036
:10A490004B2F47001C004F008300085B20557020A5
:10A4A000746F20000A00DC0C8300015D00004F0087
:10A4B000D52F4900460004000B0046009AFF0B0010
:10A4C0004800746F2D64656275672D77696E646FDF
:10A4D000770F1A30C400F401000000726573746FC6
:10A4E00072652D77696E646F770E5A30C400F8017B
:10A4F00000002E64656275672D73686F72742D6835
:10A50000656C70116630BF008300465374657070CF
:10A510006572206B6579733A203C73706163653EA8
:10A5200020446F776E20557020436F6E74696E758E
:10A530006520466F72746820476F2048656C7020F4
:10A540003F2053656520247472696E6720517569D8
:10A5500074004F004800002E64656275672D6C6FB3
:10A560006E672D68656C70107330BF0083000E4BF2
:10A5700065792020202020416374696F6E004F00B0
:10A5800083001E3C73706163653E2045786563758A
:10A59000746520646973706C6179656420776F728B
:10A5A00064004F0083002B442020202020202044E2
:10A5B0006F776E3A205374657020646F776E2069F0
:10A5C0006E746F20646973706C6179656420776F55
:10A5D000726400004F0083003C5520202020202082
:10A5E0002055703A2046696E6973682063757272EF
:10A5F000656E7420646566696E6974696F6E20614A
:10A600006E64207374657020696E206974732063B2
:10A61000616C6C6572004F0083003B43202020205A
:10A62000202020436F6E74696E75653A20747261E4
:10A6300063652063757272656E7420646566696E09
:10A640006974696F6E20776974686F7574207374AC
:10A650006F7070696E6700004F00830034462020E1
:10A660002020202020466F7274683A20656E746541
:10A67000722061207375626F7264696E6174652007
:10A68000466F72746820696E746572707265746565
:10A6900072004F00830034472020202020202047D4
:10A6A0006F3A20726573756D65206E6F726D616CA7
:10A6B00020657865637574696F6E202873746F7098
:10A6C00020646562756767696E6729004F008300C3
:10A6D00022482020202020202048656C703A2064E9
:10A6E0006973706C61792074686973206D65737328
:10A6F000616765004F0083002C3F20202020202030
:10A7000020446973706C61792073686F7274206C77
:10A71000697374206F6620646562756720636F6D6E
:10A720006D616E6473004F0083003452202020203E
:10A73000202020525354726163653A2053686F772A
:10A7400020636F6E74656E7473206F6620466F723F
:10A7500074682072657475726E20737461636B0027
:10A760004F00830030532020202020202053656597
:10A770003A204465636F6D70696C65206465666935
:10A780006E6974696F6E206265696E6720646562C8
:10A790007567676564004F00830033242020202004
:10A7A000202020446973706C617920746F70206F71
:10A7B0006620737461636B206173206164722C6C1A
:10A7C000656E207465787420737472696E6700001A
:10A7D0004F008300435C2020202020202044697308
:10A7E000706C617920466F7274682072657475723E
:10A7F0006E20737461636B206173206E756D62658A
:10A80000727320286C696B652074686520646174BC
:10A810006120737461636B2900004F008300345121
:10A8200020202020202020517569743A2061626127
:10A830006E646F6E20657865637574696F6E206FE6
:10A840006620746865206465627567676564207753
:10A850006F7264004F00830030562020202020209B
:10A860002056697375616C3A20746F67676C652058
:10A870006265747765656E20322D4420616E6420B8
:10A880007363726F6C6C696E67004F008300194CC4
:10A890002020202020202056697375616C3A207298
:10A8A00065646973706C617900004F004800006353
:10A8B0006D642D636F6C756D6E0AA530C000180055
:10A8C0000000746F2D636D642D636F6C756D6E0D7C
:10A8D0004E32BF004E32B419480000737461636B8E
:10A8E0002D6C696E650A5932C700FC0100737461F2
:10A8F000636B2D636F6C756D6E0C6432C0002D0040
:10A9000000000066756C6C2D737461636B2D780CA0
:10A910006E32C70000020066756C6C2D7374616343
:10A920006B2D790C7932C7000402726573756C74F3
:10A930002D6C696E650B8332C70008020072657367
:10A94000756C742D636F6C0A8C32C7000C02746FC7
:10A950002D737461636B2D6C6F636174696F6E111D
:10A960009532BF006E326432F21D501D480073688C
:10A970006F772D66756C6C2D737461636B0FA132EC
:10A98000BF0079328332F21D501D1D0021004700A7
:10A99000180083000F537461636B20556E646572F9
:10A9A000666C6F77000049001D00220047000E0012
:10A9B000830005456D707479000049001D00780022
:10A9C0000700200047000A008300032E2E2000000D
:10A9D0001D001D007800070006005D002C007E00B1
:10A9E00012001D00440006003D0B1200FB218000F8
:10A9F000F2FF48000073686F772D706172746961AF
:10AA00006C2D737461636B12B032BF00B032A1322F
:10AA10008300025C20001D00210047001E0083000F
:10AA20000F537461636B20556E646572666C6F774B
:10AA3000000092053000880049001D0022004700F8
:10AA40000E00830005456D707479000049001D00FB
:10AA500078000300200047000A008300032E2E2008
:10AA600000001D001D007800040006005D002C00A1
:10AA70007E0012001D00440006003D0B1200FB2169
:10AA80008000F2FF4800736176652D726573756C06
:10AA9000742D6C6F630FF532BF00B0053000750088
:10AAA0009532F90DB605300075008C32F90D48006D
:10AAB000746F2D726573756C742D6C6F630D3C3300
:10AAC000BF0095328C328E06F21DB6053500B005FA
:10AAD00035004800747279035033BF001408140025
:10AAE00047000C0053080B005706460004005E06A2
:10AAF0004800007265736F6C76652D6D6574686FC4
:10AB0000640E5D33C4001002000000657865637553
:10AB1000746572087233BF000A0075000D021F00D1
:10AB20000D00750014081F000300470006000B000D
:10AB30000A00723348002F23627566057B33C0001C
:10AB400048000000236275662D73617665098F33B6
:10AB5000B6161402000048000000912E00686C64D4
:10AB60002D73617665089833C10018020000736880
:10AB70006F772D72737461636B0BA433C1001C0279
:10AB800000006865782D737461636B09AE33C10092
:10AB900020020000736176652305B733BF00B30B55
:10ABA0008F330600983378004800A30E8A113000D6
:10ABB000A4333500480000726573746F7265230812
:10ABC000BE33BF009833B30B8F33060078004800C4
:10ABD000A30EA43330008A11350048000074686564
:10ABE0002D697006D133C7002402007468652D7288
:10ABF0007006E333C7002802007265646973706CE5
:10AC000061793F0AEA33BF00622FE3336120890A8A
:10AC1000480000282E727304F333BF00AE333000B7
:10AC2000220047000400490083000E7265747572AB
:10AC30006E2D737461636B3A20000915970530001F
:10AC4000EA33780005002E0B7E000E004400300031
:10AC50002C121F0B8100F6FF2715480073657475D1
:10AC6000702D7363726F6C6C696E672D646973709D
:10AC70006C617917FD33BF000908E33331063000FA
:10AC80001F0047000C008300023A200046000E001F
:10AC9000830007496E736964652000003106300047
:10ACA00061200A007500622FF90DDC0C480000736A
:10ACB000657475702D32642D646973706C617910E0
:10ACC0002B34BF000A1E78004E00921935007330F5
:10ACD000780046009219350083000943616C6C6569
:10ACE00072733A20000097053000EA33280BA00663
:10ACF000501D4F007800280092193500830007533B
:10AD00007461636B3A200000B00530007500793241
:10AD1000F90DB605300075008332F90D4F00E333AD
:10AD20002829E33361207500622FF90D4F00E333CA
:10AD3000BD22220047000A0075006432F90D0B00A5
:10AD4000480073657475702D64656275672D64695C
:10AD500073706C6179135134BF00F33347001600F0
:10AD60004B2F470008002B344600040051345D008F
:10AD7000AE33350048000073686F772D64656275E7
:10AD8000672D737461636B109C34BF004B2F4700B9
:10AD90005A00BE334E322600B419B7333000470094
:10ADA000040009158300022820006012B733300028
:10ADB000470004002715AE33300047000400FD3380
:10ADC000830001290000D1334F007500000C75008D
:10ADD000DD22F90DE333AE280B007500E622750085
:10ADE000DD22F90D5932460014003C33F532E333CD
:10ADF000D122B605300075006432F90D48000064B8
:10AE0000656275672D696E7465726163740EB53421
:10AE1000BF00BE339C34512F3000470004005A302D
:10AE2000B534512F30004D0003004700DC02512F94
:10AE3000490C572F410C4C000A00A5001E0047008A
:10AE400006000B00A5004B2F47000A000A004E0029
:10AE50004600040050330B166630760044000000B4
:10AE60000D001F00470014000B00E33334007B3358
:10AE70007500D52F5D3346008C027600550000002A
:10AE80000D001F00470010000B00EA3375001A3058
:10AE90005D33460070027600430000000D001F0085
:10AEA000470028000B00512F30002200512F3500A1
:10AEB000512F3000220047000C005E0675004B2F1A
:10AEC000F90D6D2F5E0646003C027600460000003C
:10AED0000D001F00470038000B004F008300235473
:10AEE0007970652027726573756D652720746F20F2
:10AEF00072657475726E20746F2064656275676721
:10AF0000657200004F00660857064600F80176009B
:10AF1000470000000D001F0047000E000B0014301A
:10AF20004F005E064600DE017600480000000D007E
:10AF30001F0047000E000B004F00A53057064600CB
:10AF4000C4017600520000000D001F0047002800D9
:10AF50000B004F008300034950200000E3332C1204
:10AF60001C002C124F0097053000EA33280B392CB7
:10AF70005706460090017600530000000D001F00A8
:10AF8000470014000B004F0031063000EE0C232266
:10AF900057064600700176003F0000000D001F00BC
:10AFA00047000E000B004F00733057064600560155
:10AFB0007600240000000D001F00470014000B0065
:10AFC000BD0B8E0650004F00593257064600360121
:10AFD0007600510000000D001F00470018000B0014
:10AFE0004F00830005756E62756700005A005E06AB
:10AFF000460012017600280000000D001F004700E7
:10B000000E000B00E333952F57064600F80076003C
:10B010003C0000000D001F00470018000B00E33348
:10B02000960C952F780001003B0635005706460028
:10B03000D4007600290000000D001F004700180012
:10B040000B00E33336063500780001003B0635007F
:10B0500057064600B00076002A0000000D001F00D1
:10B0600047001A000B00E33361200A003106350067
:10B070008C2F36063500570646008A0076005C00A5
:10B0800000000D001F00470014000B00AE3330001D
:10B090002200AE333500570646006A00760058009D
:10B0A00000000D001F00470014000B00B7333000F4
:10B0B0002200B7333500570646004A0076004C00A0
:10B0C00000000D001F0047000C000B006D2F5706FD
:10B0D000460032007600560000000D001F004700B9
:10B0E0001E000B004B2F220075004B2FF90D4B2F2C
:10B0F0002200470004006D2F5706460008005E0638
:10B100000C000B00460004005E06470008FDD1332A
:10B1100048000028747261636506F834BF001C00A3
:10B120007500E333F90D89007500EA33F90DF83441
:10B13000E33334000A00750002021F000C007500A2
:10B1400007021F000300470006004F006D2F480054
:10B150006465627567051430BF007C097330D52FB4
:10B160004800646562756767696E67099C36BF0051
:10B170007C0973300A00D52F4A00480000726573BD
:10B18000756D6506A736BF005E065E0835006D2F3B
:10B190004800007374657070696E6708B336BF004D
:10B1A000512F490C480074726163696E6707BF369E
:10B1B000BF00512F410C4800006361727265740634
:10B1C000C836C0000D000000006C696E65666565DC
:10B1D0006408D136C0000A000000006C6F673204BA
:10B1E000DA36BF005D000C002B00140047000A0097
:10B1F0000C0025004600F0FF48007363616E2D745B
:10B200006F07E136BF000D008E063100890A470046
:10B21000080025004600F2FF0E000D000600480061
:10B220006373636F756E7407F236BF005D00F236AC
:10B2300048002E63737472050537BF000537500050
:10B24000480062652D6C40050D37BF0015001700E2
:10B25000310078000800F70C1700250031000300CA
:10B2600078000800F70C1700260031000300780072
:10B270000800F70C160078000300050031000300F9
:10B28000480062652D7721051537BF008E06250021
:10B2900036000C0078000800FF0C0C003600480057
:10B2A000006C62666C6970063537BF00EF1F0C00DA
:10B2B00096060C003720480000636F6D7004453718
:10B2C000BF000F0040004800656F6C035037C70097
:10B2D0002C025C815737BF0057376100A006480039
:10B2E0006C6F61642D62617365095B37BF005E003E
:10B2F0007800005005004800006478026637BF00FF
:10B3000066374C000A0078000400890A47000C00E8
:10B310000D00360025004600EAFF0B0066370F00DF
:10B320000600480000646C026F37BF006F37B60834
:10B3300048007370696E730585370A2C00000000A1
:10B34000692D0000776669038D370A2C0100000023
:10B350002D006765742D6D736563730995370A2C2D
:10B36000020000002D6E0000006140029F370A2C91
:10B3700003000000692D6E0000702102A7370A2C1F
:10B380000400000069692D0000704002AF370A2CEC
:10B3900005000000692D6E00006D2102B7370A2CF0
:10B3A0000600000069692D006765742D757365637B
:10B3B0007309BF370A2C070000002D6E000064657A
:10B3C0006C617905CA370A2C080000006E2D000058
:10B3D00062796503D3370A2C090000002D002F6E17
:10B3E0007603DB370A2C0A0000002D6E00006E7613
:10B3F0002D6261736507E2370A2C0B0000002D6E89
:10B4000000006E762D6C656E67746809EC370A2C47
:10B410000C0000002D6E00006E764003F7370A2CFA
:10B420000D000000692D69006E762103FF370A2C9C
:10B430000E00000069692D00007764020738BF0024
:10B440005D0077000E20054035004800006D730256
:10B450000F38BF009F3705000A009F370600210004
:10B460004700F6FF0B004800007573021938BF0053
:10B47000CA3705000A00CA37060021004700F6FF58
:10B480000B00480074696D657374616D700927382D
:10B49000C7003002007428023838BF009F3775009B
:10B4A0003838F90D4800002974023D38BF009F3735
:10B4B0003838060031158300026D730048000075AE
:10B4C00028024638BF00CA3775003838F90D4800E1
:10B4D000002975025238BF00CA37383806003115C6
:10B4E0008300027573004800706F72742D6123072A
:10B4F0005B38C00000000000706F72742D6223077B
:10B500006938C00001000000706F72742D6323075A
:10B510007138C00002000000706F72742D64230740
:10B520007938C00003000000706F72742D65230726
:10B530008138C00004000000007063722D626173E6
:10B5400065088938C000009004402F7063722D7028
:10B550006F7274099238C0000010000000706F72A2
:10B56000742E70696E3E7063720C9B38BF00780059
:10B57000040007000C009B38070092380500050006
:10B580004800706F72743E6770637209A638BF001E
:10B590009B380700923805007800800005004800BD
:10B5A000002B61663104B738BF007800000103004A
:10B5B0004800002B61663204C438BF0078000002E6
:10B5C00003004800002B64736504CD38BF00780089
:10B5D000400003004800002B6F646504D638BF00AC
:10B5E0007800200003004800007063722104DF38F7
:10B5F000BF00A63835004800007063724004E83888
:10B60000BF00A63830004800006932632D626173C4
:10B610006508F038C7003402006932632D73657421
:10B620002D6D6F64756C650EFA38BF0078000010E0
:10B63000070077000060064005007500FA38F90D34
:10B6400048000069326340040539BF00FA3805003C
:10B65000310048000069326321041539BF00FA380F
:10B6600005003600480073696D5F736367633409D2
:10B670001E39C00034800440006932632D636C6B56
:10B680002D6F6E2D300C2939BF002939300078001C
:10B6900040000300293935004800006932632D63FA
:10B6A0006C6B2D6F6E2D310C3439BF002939300091
:10B6B00078008000030029393500480000693263B2
:10B6C0002D7365742D70696E732D300E4539BF0072
:10B6D0005D00CD38713878000200E8385D00CD3863
:10B6E000713878000300E8384800006932632D7330
:10B6F00065742D70696E732D310E5739BF005D0072
:10B70000CD38793878000A00E8385D00CD387938CE
:10B7100078000B00E8384800006932632D736574C7
:10B720002D726174650C6E39BF005D0078000100F8
:10B730001E394800006932632D696963656E2D6F9B
:10B740006E0C8439BF007800020015397800800043
:10B750000300780002001E3948006932632D6969D0
:10B7600063656E2D6F66660D9239BF00780002002A
:10B77000153978007FFF0200780002001E3948006A
:10B78000006932632D6D73742D6F6E0AA539BF0089
:10B7900078000200153978002000030078000200CC
:10B7A0001E3948006932632D6D73742D6F66660B08
:10B7B000B739BF007800020015397800DFFF0200BA
:10B7C000780002001E3948006932632D74782D6FAD
:10B7D0006E09C939BF0078000200153978001000E1
:10B7E0000300780002001E394800006932632D749E
:10B7F000782D6F66660ADA39BF00780002001539C5
:10B800007800EFFF0200780002001E39480000694E
:10B8100032632D7478616B08EC39BF007800020048
:10B820001539780008000300780002001E3948002E
:10B83000006932632D7273746108FD39BF007800AE
:10B8400002001539780004000300780002001E3958
:10B850004800006932632D69696369663F0A0E3AE0
:10B86000BF007800030015390A00780010000200BC
:10B870004700240078001000780003001E390B00F8
:10B880005E066F0F106172626974726174696F6E27
:10B89000206C6F73740078000200020047001200F1
:10B8A00078000200780003001E395E06460004009E
:10B8B000570648006932632D776169742D6E6F2DCC
:10B8C00061636B0F203ABF0078000A009F370500C4
:10B8D0000A009F37060021006F0F0774696D656FBE
:10B8E00075740000203A4700E8FF0B00480000692B
:10B8F00032632D776169742D61636B0C533ABF001D
:10B90000533A7800030015397800010002006F0FE8
:10B91000136D697373696E672061636B6E6F776C0B
:10B9200065646765000048006932632D70757407AF
:10B930006F3ABF00780004001E396F3A4800693240
:10B94000632D67657407893ABF00780004001539D4
:10B95000533A4800006932632D6164647208943A76
:10B96000C7003802006932632D7265674008A03A4B
:10B97000BF00DA39B739A03A893A893A0E3AA03A83
:10B980002500893AEC39FD39943A0B00943AC939CB
:10B990004800006932632D7265672108A83ABF002C
:10B9A000DA39B739A03A893A893A893AC939480027
:10B9B000006932632D6F70656E08BF3ABF00450B9A
:10B9C0007500A03AF90D3439573984399239480055
:10B9D0006932632D636C6F736509CE3ABF00A53978
:10B9E00048006770696F2D6261736509DE3AC000B7
:10B9F00000F00F4000706F72742E70696E3E6D61C2
:10BA0000736B2E6770696F12E73ABF007800010010
:10BA10000C0008000C00780040000700E73A050021
:10BA20004800006770696F2D73657408F53ABF00B0
:10BA3000F53A780004000500350048000067706999
:10BA40006F2D636C7208073BBF00F53A7800080061
:10BA50000500350048006770696F2D746F67676C6B
:10BA6000650B143BBF00F53A78000C00050035006B
:10BA700048006770696F2D70696E4009223BBF00F6
:10BA8000F53A78001000050030000200950B4800E0
:10BA9000006770696F2D6469722D6F75740C2F3B90
:10BAA000BF00F53A0A0015003000030016007800C8
:10BAB00014000500350048006770696F2D646972D5
:10BAC0002D696E0B403BBF00F53A0A0015003000AF
:10BAD0000C0001000200160078001400050035007B
:10BAE00048006770696F2D6F75743F09533BBF0045
:10BAF000F53A78001400050030000200950B48006C
:10BB00002E642503673BBF001915181250007600FC
:10BB1000250000004E0027154800002E7573616750
:10BB20006506733BBF00F737780064000700E23713
:10BB30008D00733B48006E762403823BBF00EC37D8
:10BB4000F73748002E6E76038E3BBF008E3B5000C9
:10BB500048006E762D64756D7007953BBF008E3B77
:10BB60002500BE1248006E762D64756D702D616CD7
:10BB70006C0B9E3BBF00EC37E237371B48006E76FC
:10BB80002D6576616C756174650BAA3BBF008E3BB9
:10BB90007500B6081408140047000400FF1448009C
:10BBA000006E7602B63BBF00F737573761000A00D8
:10BBB000220047000600FF144900570E7F001000C6
:10BBC000440031000D00073825008000F4FF7800A4
:10BBD0000A000D00073825005D000C0007384800FA
:10BBE00000737472726E6C06C33BBF000C007F0062
:10BBF0001C004400310078000A001F0047000600C6
:10BC000044007D007800FFFF8100E8FF48006E7669
:10BC10002D756E646F07E53BBF008E3B27000A0061
:10BC2000210047001200A0068300076E6F206D6F91
:10BC3000726500004900570EE53BEC370600250011
:10BC40005D000C00073848006E762D776970650737
:10BC5000FC3BBF005D005D000738480062652D6950
:10BC60006E05193CBF005D000C00BF374800006244
:10BC7000652D6F757406223CBF00780001000C0032
:10BC8000BF37480062652D70756C6C7570092C3C6F
:10BC9000BF00780002000C00BF374800676F2D6FAF
:10BCA0006E05383CBF00780001000C00AF3748003B
:10BCB00000676F2D6F666606423CBF005D000C009A
:10BCC000AF3748000077616974044D3CBF009F376F
:10BCD00005000A009F37060021004D0003004700C1
:10BCE000F2FF0B004800006C6202563CBF00780077
:10BCF0000D002C3C78000E002C3C78000D00423CDE
:10BD000078007D00563C78000D004D3C78000E0018
:10BD1000423C78007D00563C78000E004D3C4D00C2
:10BD20004700D8FF4800002E74736C04663CBF00C7
:10BD300078003900CE3A7800030078008000BF3ADE
:10BD400078009201193878008C00A83A78008D00AC
:10BD5000A83A4A202C1278008E00A83A78008F006A
:10BD6000A83A4A202C125D0078008000BF3ADE3AE3
:10BD7000480000676F02873CBF0078000100780030
:10BD80000D00BF377800010078000D00AF37780054
:10BD90000A0019387800000078000D00AF377800ED
:10BDA000000078000D00BF37480000636F6E6669C1
:10BDB000726D3F08AC3CBF007800000078000D00B9
:10BDC000BF377800010078000D00AF37780002001F
:10BDD000193878000D00B7377800010078000D00A1
:10BDE000BF377800000078000D00AF374800617061
:10BDF0007003CB3CBF00CB3C47000600AC3CB63BDD
:10BE000083000643466F727468004F001709950857
:10BE10004800FFFFCD050000B9050000C105000086
:10BE200095120000C515000005160000211600003F
:10BE300059160000951600006D070000CD16000091
:10BE4000451700004D17000091170000B9170000BA
:10BE5000FFFFFFFF1201000202000040C016830432
:10BE600000010102030118035400650065006E0023
:10BE7000730079006400750069006E006F000902AC
:10BE80004300020100C03209040000010202010067
:10BE900005240010010524010101042402060524E3
:10BEA0000600010705820310004009040100020A90
:10BEB000000000070503024000000705840240005F
:10BEC0000000160355005300420020005300650097
:10BED0007200690061006C00040309040C03000097
:10BEE0000000000000000000000000000000000052
:04BEF00000000A0440
:00000001FF
